
 Start         Length     Name                   Class
 0001:00401000 000219D8H .text                   CODE
 0002:00423000 000003C8H .itext                  ICODE
 0003:00424000 00000064H .data                   DATA
 0004:00425000 000000ACH .bss                    BSS
 0005:00000000 00000000H .tls                    TLS


Detailed map of segments

 0001:00000000 000001F6 C=CODE     S=.text    G=(none)   M=System   ACBP=A9
 0001:000001F8 00000006 C=CODE     S=.text    G=(none)   M=ShellAPI ACBP=A9
 0001:00000200 00000074 C=CODE     S=.text    G=(none)   M=Windows  ACBP=A9
 0001:00000274 00000066 C=CODE     S=.text    G=(none)   M=SysUtils ACBP=A9
 0001:000002DC 000000DE C=CODE     S=.text    G=(none)   M=StdCtrls ACBP=A9
 0001:000003BC 00000006 C=CODE     S=.text    G=(none)   M=ActnList ACBP=A9
 0001:000003C4 000000D6 C=CODE     S=.text    G=(none)   M=Classes  ACBP=A9
 0001:0000049C 00000016 C=CODE     S=.text    G=(none)   M=TypInfo  ACBP=A9
 0001:000004B4 00000006 C=CODE     S=.text    G=(none)   M=Variants ACBP=A9
 0001:000004BC 00000006 C=CODE     S=.text    G=(none)   M=VarUtils ACBP=A9
 0001:000004C4 00000016 C=CODE     S=.text    G=(none)   M=ImgList  ACBP=A9
 0001:000004DC 000000C6 C=CODE     S=.text    G=(none)   M=Graphics ACBP=A9
 0001:000005A4 00000006 C=CODE     S=.text    G=(none)   M=Registry ACBP=A9
 0001:000005AC 0000000E C=CODE     S=.text    G=(none)   M=IniFiles ACBP=A9
 0001:000005BC 00000006 C=CODE     S=.text    G=(none)   M=Themes   ACBP=A9
 0001:000005C4 0000029E C=CODE     S=.text    G=(none)   M=Controls ACBP=A9
 0001:00000864 00000016 C=CODE     S=.text    G=(none)   M=Menus    ACBP=A9
 0001:0000087C 00000006 C=CODE     S=.text    G=(none)   M=UxTheme  ACBP=A9
 0001:00000884 00000006 C=CODE     S=.text    G=(none)   M=MultiMon ACBP=A9
 0001:0000088C 00000006 C=CODE     S=.text    G=(none)   M=DwmApi   ACBP=A9
 0001:00000894 00000176 C=CODE     S=.text    G=(none)   M=Forms    ACBP=A9
 0001:00000A0C 00000006 C=CODE     S=.text    G=(none)   M=HelpIntfs ACBP=A9
 0001:00000A14 0000003E C=CODE     S=.text    G=(none)   M=Dialogs  ACBP=A9
 0001:00000A54 00000006 C=CODE     S=.text    G=(none)   M=Printers ACBP=A9
 0001:00000A5C 00000016 C=CODE     S=.text    G=(none)   M=ExtCtrls ACBP=A9
 0001:00000A74 00000006 C=CODE     S=.text    G=(none)   M=GraphUtil ACBP=A9
 0001:00000A7C 00000016 C=CODE     S=.text    G=(none)   M=Clipbrd  ACBP=A9
 0001:00000A94 00000006 C=CODE     S=.text    G=(none)   M=FlatSB   ACBP=A9
 0001:00000A9C 000001D6 C=CODE     S=.text    G=(none)   M=DesignEditors ACBP=A9
 0001:00000C74 0000002E C=CODE     S=.text    G=(none)   M=DesignIntf ACBP=A9
 0001:00000CA4 00000006 C=CODE     S=.text    G=(none)   M=ToolsAPI ACBP=A9
 0001:00000CAC 00000006 C=CODE     S=.text    G=(none)   M=XMLIntf  ACBP=A9
 0001:00000CB4 00000006 C=CODE     S=.text    G=(none)   M=xmldom   ACBP=A9
 0001:00000CBC 00000006 C=CODE     S=.text    G=(none)   M=msxmldom ACBP=A9
 0001:00000CC4 00000006 C=CODE     S=.text    G=(none)   M=ComObj   ACBP=A9
 0001:00000CCC 0000006E C=CODE     S=.text    G=(none)   M=ComCtrls ACBP=A9
 0001:00000D3C 00000006 C=CODE     S=.text    G=(none)   M=ExtActns ACBP=A9
 0001:00000D44 00000006 C=CODE     S=.text    G=(none)   M=ExtDlgs  ACBP=A9
 0001:00000D4C 00000006 C=CODE     S=.text    G=(none)   M=Buttons  ACBP=A9
 0001:00000D54 00000006 C=CODE     S=.text    G=(none)   M=Mapi     ACBP=A9
 0001:00000D5C 00000006 C=CODE     S=.text    G=(none)   M=DockForm ACBP=A9
 0001:00000D64 00000006 C=CODE     S=.text    G=(none)   M=IDEMessages ACBP=A9
 0001:00000D6C 00000006 C=CODE     S=.text    G=(none)   M=DeskForm ACBP=A9
 0001:00000D74 00000006 C=CODE     S=.text    G=(none)   M=BaseDock ACBP=A9
 0001:00000D7C 00000006 C=CODE     S=.text    G=(none)   M=PercentageDockTree ACBP=A9
 0001:00000D84 00000006 C=CODE     S=.text    G=(none)   M=CaptionedDockTree ACBP=A9
 0001:00000D8C 00000006 C=CODE     S=.text    G=(none)   M=DockTabSet ACBP=A9
 0001:00000D94 00000006 C=CODE     S=.text    G=(none)   M=Tabs     ACBP=A9
 0001:00000D9C 00000006 C=CODE     S=.text    G=(none)   M=DeskUtil ACBP=A9
 0001:00000DA4 00000006 C=CODE     S=.text    G=(none)   M=ActnMan  ACBP=A9
 0001:00000DAC 00000006 C=CODE     S=.text    G=(none)   M=ActnMenus ACBP=A9
 0001:00000DB4 00000006 C=CODE     S=.text    G=(none)   M=XPStyleActnCtrls ACBP=A9
 0001:00000DBC 00000006 C=CODE     S=.text    G=(none)   M=Proxies  ACBP=A9
 0001:00000DC4 00000056 C=CODE     S=.text    G=(none)   M=ovccmd   ACBP=A9
 0001:00000E1C 00000016 C=CODE     S=.text    G=(none)   M=ovcmisc  ACBP=A9
 0001:00000E34 0000000E C=CODE     S=.text    G=(none)   M=ovcdata  ACBP=A9
 0001:00000E44 00000006 C=CODE     S=.text    G=(none)   M=o32sr    ACBP=A9
 0001:00000E4C 00000006 C=CODE     S=.text    G=(none)   M=ovcdate  ACBP=A9
 0001:00000E54 00000006 C=CODE     S=.text    G=(none)   M=ovcstr   ACBP=A9
 0001:00000E5C 000000AE C=CODE     S=.text    G=(none)   M=ovcbase  ACBP=A9
 0001:00000F0C 00000016 C=CODE     S=.text    G=(none)   M=ovcintl  ACBP=A9
 0001:00000F24 0000012E C=CODE     S=.text    G=(none)   M=ovcef    ACBP=A9
 0001:00001054 00000006 C=CODE     S=.text    G=(none)   M=ovccalc  ACBP=A9
 0001:0000105C 00000006 C=CODE     S=.text    G=(none)   M=ovcuser  ACBP=A9
 0001:00001064 00000066 C=CODE     S=.text    G=(none)   M=ovcae    ACBP=A9
 0001:000010CC 0000001E C=CODE     S=.text    G=(none)   M=VCLEditors ACBP=A9
 0001:000010EC 00000026 C=CODE     S=.text    G=(none)   M=ovcdrpvw ACBP=A9
 0001:00001114 0000003E C=CODE     S=.text    G=(none)   M=ovcfiler ACBP=A9
 0001:00001154 000000BE C=CODE     S=.text    G=(none)   M=ovcrptvw ACBP=A9
 0001:00001214 00000006 C=CODE     S=.text    G=(none)   M=ovcrvexpdef ACBP=A9
 0001:0000121C 00000016 C=CODE     S=.text    G=(none)   M=ovcrvidx ACBP=A9
 0001:00001234 0000003E C=CODE     S=.text    G=(none)   M=Grids    ACBP=A9
 0001:00001274 0000000E C=CODE     S=.text    G=(none)   M=ovcfxfnt ACBP=A9
 0001:00001284 0000006E C=CODE     S=.text    G=(none)   M=ovclabel ACBP=A9
 0001:000012F4 0000000E C=CODE     S=.text    G=(none)   M=ovcclrcb ACBP=A9
 0001:00001304 00000026 C=CODE     S=.text    G=(none)   M=ovclkout ACBP=A9
 0001:0000132C 00000006 C=CODE     S=.text    G=(none)   M=ovcstate ACBP=A9
 0001:00001334 0000000E C=CODE     S=.text    G=(none)   M=ovcnbk   ACBP=A9
 0001:00001344 0000000E C=CODE     S=.text    G=(none)   M=ovctcnum ACBP=A9
 0001:00001354 00000076 C=CODE     S=.text    G=(none)   M=ovctcbef ACBP=A9
 0001:000013CC 00000046 C=CODE     S=.text    G=(none)   M=ovctcell ACBP=A9
 0001:00001414 0000003E C=CODE     S=.text    G=(none)   M=ovctbcls ACBP=A9
 0001:00001454 0000003E C=CODE     S=.text    G=(none)   M=ovctbrws ACBP=A9
 0001:00001494 0000001E C=CODE     S=.text    G=(none)   M=ovcedsld ACBP=A9
 0001:000014B4 0000004E C=CODE     S=.text    G=(none)   M=ovcoutln ACBP=A9
 0001:00001504 00000006 C=CODE     S=.text    G=(none)   M=o32vldtr ACBP=A9
 0001:0000150C 00000006 C=CODE     S=.text    G=(none)   M=o32rxvld ACBP=A9
 0001:00001514 0000000E C=CODE     S=.text    G=(none)   M=o32vlreg ACBP=A9
 0001:00001524 00000006 C=CODE     S=.text    G=(none)   M=o32pvldr ACBP=A9
 0001:0000152C 00000006 C=CODE     S=.text    G=(none)   M=o32ovldr ACBP=A9
 0001:00001534 000000A6 C=CODE     S=.text    G=(none)   M=o32igrid ACBP=A9
 0001:000015DC 0000000E C=CODE     S=.text    G=(none)   M=ovcftcbx ACBP=A9
 0001:000015EC 00000006 C=CODE     S=.text    G=(none)   M=OvcUtils ACBP=A9
 0001:000015F4 0000000E C=CODE     S=.text    G=(none)   M=o32flxbn ACBP=A9
 0001:00001604 00000006 C=CODE     S=.text    G=(none)   M=O32MouseMon ACBP=A9
 0001:0000160C 00000016 C=CODE     S=.text    G=(none)   M=CheckLst ACBP=A9
 0001:00001624 0000002E C=CODE     S=.text    G=(none)   M=o32lkout ACBP=A9
 0001:00001654 0000000E C=CODE     S=.text    G=(none)   M=ovclb    ACBP=A9
 0001:00001664 0000000E C=CODE     S=.text    G=(none)   M=ovctcpic ACBP=A9
 0001:00001674 0000000E C=CODE     S=.text    G=(none)   M=ovctcsim ACBP=A9
 0001:00001684 00000006 C=CODE     S=.text    G=(none)   M=ovctgres ACBP=A9
 0001:0000168C 00000006 C=CODE     S=.text    G=(none)   M=ovcplb   ACBP=A9
 0001:00001694 00000006 C=CODE     S=.text    G=(none)   M=ovcxfer  ACBP=A9
 0001:0000169C 000001C3 C=CODE     S=.text    G=(none)   M=SysInit  ACBP=A9
 0001:00001860 0000067A C=CODE     S=.text    G=(none)   M=Ovcabot0 ACBP=A9
 0001:00001EDC 00000B9A C=CODE     S=.text    G=(none)   M=ovcaepe  ACBP=A9
 0001:00002A78 0000122A C=CODE     S=.text    G=(none)   M=ovccole0 ACBP=A9
 0001:00003CA4 00000186 C=CODE     S=.text    G=(none)   M=ovcbtnh0 ACBP=A9
 0001:00003E2C 0000035E C=CODE     S=.text    G=(none)   M=ovccmdp1 ACBP=A9
 0001:0000418C 00001FFE C=CODE     S=.text    G=(none)   M=ovccmdp0 ACBP=A9
 0001:0000618C 000002C2 C=CODE     S=.text    G=(none)   M=ovccolr0 ACBP=A9
 0001:00006450 00000656 C=CODE     S=.text    G=(none)   M=ovcdock0 ACBP=A9
 0001:00006AA8 00000886 C=CODE     S=.text    G=(none)   M=Ovcdrpve ACBP=A9
 0001:00007330 00000AE2 C=CODE     S=.text    G=(none)   M=OvcEfPe  ACBP=A9
 0001:00007E14 000002AE C=CODE     S=.text    G=(none)   M=ovcfnpe  ACBP=A9
 0001:000080C4 0000033E C=CODE     S=.text    G=(none)   M=ovcfxfpe ACBP=A9
 0001:00008404 00000A66 C=CODE     S=.text    G=(none)   M=ovclbl2  ACBP=A9
 0001:00008E6C 0000025E C=CODE     S=.text    G=(none)   M=ovclbl1  ACBP=A9
 0001:000090CC 0000245E C=CODE     S=.text    G=(none)   M=ovclbl0  ACBP=A9
 0001:0000B52C 00000F0A C=CODE     S=.text    G=(none)   M=ovclkou1 ACBP=A9
 0001:0000C438 000001E6 C=CODE     S=.text    G=(none)   M=ovclkou0 ACBP=A9
 0001:0000C620 00000176 C=CODE     S=.text    G=(none)   M=ovcnbk0  ACBP=A9
 0001:0000C798 00000896 C=CODE     S=.text    G=(none)   M=OvcNfPe  ACBP=A9
 0001:0000D030 00000CD2 C=CODE     S=.text    G=(none)   M=Ovcoutle ACBP=A9
 0001:0000DD04 00000CC6 C=CODE     S=.text    G=(none)   M=o32vldpe ACBP=A9
 0001:0000E9CC 00002636 C=CODE     S=.text    G=(none)   M=O32IGridEditor1 ACBP=A9
 0001:00011004 0000110A C=CODE     S=.text    G=(none)   M=o32coled ACBP=A9
 0001:00012110 000010BA C=CODE     S=.text    G=(none)   M=O32LobEd ACBP=A9
 0001:000131CC 000010AA C=CODE     S=.text    G=(none)   M=O32IGridItemEd ACBP=A9
 0001:00014278 00000DB2 C=CODE     S=.text    G=(none)   M=ovcrvped ACBP=A9
 0001:0001502C 0000347A C=CODE     S=.text    G=(none)   M=ovcrvced ACBP=A9
 0001:000184A8 00000B92 C=CODE     S=.text    G=(none)   M=ovctcpe  ACBP=A9
 0001:0001903C 00000A6E C=CODE     S=.text    G=(none)   M=ovctbpe2 ACBP=A9
 0001:00019AAC 00000A86 C=CODE     S=.text    G=(none)   M=ovctbpe1 ACBP=A9
 0001:0001A534 00001AB2 C=CODE     S=.text    G=(none)   M=ovcstat0 ACBP=A9
 0001:0001BFE8 0000230A C=CODE     S=.text    G=(none)   M=ovcxfrc1 ACBP=A9
 0001:0001E2F4 00000332 C=CODE     S=.text    G=(none)   M=ovcxfrc0 ACBP=A9
 0001:0001E628 000009A6 C=CODE     S=.text    G=(none)   M=ovcpfpe  ACBP=A9
 0001:0001EFD0 0000074E C=CODE     S=.text    G=(none)   M=OvcSfPe  ACBP=A9
 0001:0001F720 000019A6 C=CODE     S=.text    G=(none)   M=ovcreg   ACBP=A9
 0001:000210C8 0000090F C=CODE     S=.text    G=(none)   M=.O406_d2005 ACBP=A9
 0002:00000000 00000006 C=ICODE    S=.itext   G=(none)   M=System   ACBP=A9
 0002:00000008 00000011 C=ICODE    S=.itext   G=(none)   M=Windows  ACBP=A9
 0002:0000001C 00000006 C=ICODE    S=.itext   G=(none)   M=SysUtils ACBP=A9
 0002:00000024 00000006 C=ICODE    S=.itext   G=(none)   M=ActnList ACBP=A9
 0002:0000002C 00000006 C=ICODE    S=.itext   G=(none)   M=Classes  ACBP=A9
 0002:00000034 00000006 C=ICODE    S=.itext   G=(none)   M=TypInfo  ACBP=A9
 0002:0000003C 00000006 C=ICODE    S=.itext   G=(none)   M=Variants ACBP=A9
 0002:00000044 00000006 C=ICODE    S=.itext   G=(none)   M=VarUtils ACBP=A9
 0002:0000004C 00000006 C=ICODE    S=.itext   G=(none)   M=Graphics ACBP=A9
 0002:00000054 00000006 C=ICODE    S=.itext   G=(none)   M=Registry ACBP=A9
 0002:0000005C 00000006 C=ICODE    S=.itext   G=(none)   M=IniFiles ACBP=A9
 0002:00000064 00000006 C=ICODE    S=.itext   G=(none)   M=Themes   ACBP=A9
 0002:0000006C 00000006 C=ICODE    S=.itext   G=(none)   M=Controls ACBP=A9
 0002:00000074 00000006 C=ICODE    S=.itext   G=(none)   M=Menus    ACBP=A9
 0002:0000007C 00000006 C=ICODE    S=.itext   G=(none)   M=UxTheme  ACBP=A9
 0002:00000084 00000006 C=ICODE    S=.itext   G=(none)   M=MultiMon ACBP=A9
 0002:0000008C 00000006 C=ICODE    S=.itext   G=(none)   M=DwmApi   ACBP=A9
 0002:00000094 00000006 C=ICODE    S=.itext   G=(none)   M=Forms    ACBP=A9
 0002:0000009C 00000006 C=ICODE    S=.itext   G=(none)   M=HelpIntfs ACBP=A9
 0002:000000A4 00000006 C=ICODE    S=.itext   G=(none)   M=Dialogs  ACBP=A9
 0002:000000AC 00000006 C=ICODE    S=.itext   G=(none)   M=Printers ACBP=A9
 0002:000000B4 00000006 C=ICODE    S=.itext   G=(none)   M=ExtCtrls ACBP=A9
 0002:000000BC 00000006 C=ICODE    S=.itext   G=(none)   M=GraphUtil ACBP=A9
 0002:000000C4 00000006 C=ICODE    S=.itext   G=(none)   M=Clipbrd  ACBP=A9
 0002:000000CC 00000006 C=ICODE    S=.itext   G=(none)   M=FlatSB   ACBP=A9
 0002:000000D4 00000006 C=ICODE    S=.itext   G=(none)   M=DesignEditors ACBP=A9
 0002:000000DC 00000006 C=ICODE    S=.itext   G=(none)   M=ToolsAPI ACBP=A9
 0002:000000E4 00000006 C=ICODE    S=.itext   G=(none)   M=XMLIntf  ACBP=A9
 0002:000000EC 00000006 C=ICODE    S=.itext   G=(none)   M=xmldom   ACBP=A9
 0002:000000F4 00000006 C=ICODE    S=.itext   G=(none)   M=msxmldom ACBP=A9
 0002:000000FC 00000006 C=ICODE    S=.itext   G=(none)   M=ComObj   ACBP=A9
 0002:00000104 00000006 C=ICODE    S=.itext   G=(none)   M=ComCtrls ACBP=A9
 0002:0000010C 00000006 C=ICODE    S=.itext   G=(none)   M=ExtActns ACBP=A9
 0002:00000114 00000006 C=ICODE    S=.itext   G=(none)   M=ExtDlgs  ACBP=A9
 0002:0000011C 00000006 C=ICODE    S=.itext   G=(none)   M=Buttons  ACBP=A9
 0002:00000124 00000006 C=ICODE    S=.itext   G=(none)   M=Mapi     ACBP=A9
 0002:0000012C 00000006 C=ICODE    S=.itext   G=(none)   M=DockForm ACBP=A9
 0002:00000134 00000006 C=ICODE    S=.itext   G=(none)   M=IDEMessages ACBP=A9
 0002:0000013C 00000006 C=ICODE    S=.itext   G=(none)   M=DeskForm ACBP=A9
 0002:00000144 00000006 C=ICODE    S=.itext   G=(none)   M=BaseDock ACBP=A9
 0002:0000014C 00000006 C=ICODE    S=.itext   G=(none)   M=PercentageDockTree ACBP=A9
 0002:00000154 00000006 C=ICODE    S=.itext   G=(none)   M=CaptionedDockTree ACBP=A9
 0002:0000015C 00000006 C=ICODE    S=.itext   G=(none)   M=DockTabSet ACBP=A9
 0002:00000164 00000006 C=ICODE    S=.itext   G=(none)   M=Tabs     ACBP=A9
 0002:0000016C 00000006 C=ICODE    S=.itext   G=(none)   M=DeskUtil ACBP=A9
 0002:00000174 00000006 C=ICODE    S=.itext   G=(none)   M=ActnMan  ACBP=A9
 0002:0000017C 00000006 C=ICODE    S=.itext   G=(none)   M=ActnMenus ACBP=A9
 0002:00000184 00000006 C=ICODE    S=.itext   G=(none)   M=XPStyleActnCtrls ACBP=A9
 0002:0000018C 00000006 C=ICODE    S=.itext   G=(none)   M=Proxies  ACBP=A9
 0002:00000194 00000006 C=ICODE    S=.itext   G=(none)   M=ovcdata  ACBP=A9
 0002:0000019C 00000006 C=ICODE    S=.itext   G=(none)   M=o32sr    ACBP=A9
 0002:000001A4 00000006 C=ICODE    S=.itext   G=(none)   M=ovcdate  ACBP=A9
 0002:000001AC 00000006 C=ICODE    S=.itext   G=(none)   M=ovcbase  ACBP=A9
 0002:000001B4 00000006 C=ICODE    S=.itext   G=(none)   M=ovcintl  ACBP=A9
 0002:000001BC 00000006 C=ICODE    S=.itext   G=(none)   M=ovccalc  ACBP=A9
 0002:000001C4 00000006 C=ICODE    S=.itext   G=(none)   M=ovcuser  ACBP=A9
 0002:000001CC 00000006 C=ICODE    S=.itext   G=(none)   M=VCLEditors ACBP=A9
 0002:000001D4 00000006 C=ICODE    S=.itext   G=(none)   M=ovcrptvw ACBP=A9
 0002:000001DC 00000006 C=ICODE    S=.itext   G=(none)   M=ovcrvexpdef ACBP=A9
 0002:000001E4 00000006 C=ICODE    S=.itext   G=(none)   M=ovcfxfnt ACBP=A9
 0002:000001EC 00000006 C=ICODE    S=.itext   G=(none)   M=ovcoutln ACBP=A9
 0002:000001F4 00000006 C=ICODE    S=.itext   G=(none)   M=o32rxvld ACBP=A9
 0002:000001FC 00000006 C=ICODE    S=.itext   G=(none)   M=o32vlreg ACBP=A9
 0002:00000204 00000006 C=ICODE    S=.itext   G=(none)   M=o32pvldr ACBP=A9
 0002:0000020C 00000006 C=ICODE    S=.itext   G=(none)   M=o32ovldr ACBP=A9
 0002:00000214 00000006 C=ICODE    S=.itext   G=(none)   M=O32MouseMon ACBP=A9
 0002:0000021C 00000006 C=ICODE    S=.itext   G=(none)   M=CheckLst ACBP=A9
 0002:00000224 00000006 C=ICODE    S=.itext   G=(none)   M=ovctgres ACBP=A9
 0002:0000022C 00000008 C=ICODE    S=.itext   G=(none)   M=Ovcabot0 ACBP=A9
 0002:00000234 00000008 C=ICODE    S=.itext   G=(none)   M=ovcaepe  ACBP=A9
 0002:0000023C 00000008 C=ICODE    S=.itext   G=(none)   M=ovccole0 ACBP=A9
 0002:00000244 00000008 C=ICODE    S=.itext   G=(none)   M=ovcbtnh0 ACBP=A9
 0002:0000024C 00000008 C=ICODE    S=.itext   G=(none)   M=ovccmdp1 ACBP=A9
 0002:00000254 00000008 C=ICODE    S=.itext   G=(none)   M=ovccmdp0 ACBP=A9
 0002:0000025C 00000008 C=ICODE    S=.itext   G=(none)   M=ovccolr0 ACBP=A9
 0002:00000264 00000008 C=ICODE    S=.itext   G=(none)   M=ovcdock0 ACBP=A9
 0002:0000026C 00000008 C=ICODE    S=.itext   G=(none)   M=Ovcdrpve ACBP=A9
 0002:00000274 00000008 C=ICODE    S=.itext   G=(none)   M=OvcEfPe  ACBP=A9
 0002:0000027C 00000008 C=ICODE    S=.itext   G=(none)   M=ovcfnpe  ACBP=A9
 0002:00000284 00000008 C=ICODE    S=.itext   G=(none)   M=ovcfxfpe ACBP=A9
 0002:0000028C 0000007A C=ICODE    S=.itext   G=(none)   M=ovclbl2  ACBP=A9
 0002:00000308 00000008 C=ICODE    S=.itext   G=(none)   M=ovclbl1  ACBP=A9
 0002:00000310 00000008 C=ICODE    S=.itext   G=(none)   M=ovclbl0  ACBP=A9
 0002:00000318 00000008 C=ICODE    S=.itext   G=(none)   M=ovclkou1 ACBP=A9
 0002:00000320 00000008 C=ICODE    S=.itext   G=(none)   M=ovclkou0 ACBP=A9
 0002:00000328 00000008 C=ICODE    S=.itext   G=(none)   M=ovcnbk0  ACBP=A9
 0002:00000330 00000008 C=ICODE    S=.itext   G=(none)   M=OvcNfPe  ACBP=A9
 0002:00000338 00000008 C=ICODE    S=.itext   G=(none)   M=Ovcoutle ACBP=A9
 0002:00000340 00000008 C=ICODE    S=.itext   G=(none)   M=o32vldpe ACBP=A9
 0002:00000348 00000008 C=ICODE    S=.itext   G=(none)   M=O32IGridEditor1 ACBP=A9
 0002:00000350 00000008 C=ICODE    S=.itext   G=(none)   M=o32coled ACBP=A9
 0002:00000358 00000008 C=ICODE    S=.itext   G=(none)   M=O32LobEd ACBP=A9
 0002:00000360 00000008 C=ICODE    S=.itext   G=(none)   M=O32IGridItemEd ACBP=A9
 0002:00000368 00000008 C=ICODE    S=.itext   G=(none)   M=ovcrvped ACBP=A9
 0002:00000370 00000008 C=ICODE    S=.itext   G=(none)   M=ovcrvced ACBP=A9
 0002:00000378 00000008 C=ICODE    S=.itext   G=(none)   M=ovctcpe  ACBP=A9
 0002:00000380 00000008 C=ICODE    S=.itext   G=(none)   M=ovctbpe2 ACBP=A9
 0002:00000388 00000008 C=ICODE    S=.itext   G=(none)   M=ovctbpe1 ACBP=A9
 0002:00000390 00000008 C=ICODE    S=.itext   G=(none)   M=ovcstat0 ACBP=A9
 0002:00000398 00000008 C=ICODE    S=.itext   G=(none)   M=ovcxfrc1 ACBP=A9
 0002:000003A0 00000008 C=ICODE    S=.itext   G=(none)   M=ovcxfrc0 ACBP=A9
 0002:000003A8 00000008 C=ICODE    S=.itext   G=(none)   M=ovcpfpe  ACBP=A9
 0002:000003B0 00000008 C=ICODE    S=.itext   G=(none)   M=OvcSfPe  ACBP=A9
 0002:000003B8 00000008 C=ICODE    S=.itext   G=(none)   M=ovcreg   ACBP=A9
 0002:000003C0 00000005 C=ICODE    S=.itext   G=(none)   M=.O406_d2005 ACBP=A9
 0003:00000000 0000002C C=DATA     S=.data    G=DGROUP   M=SysInit  ACBP=A9
 0003:0000002C 00000002 C=DATA     S=.data    G=DGROUP   M=ovccmdp0 ACBP=A9
 0003:00000030 00000018 C=DATA     S=.data    G=DGROUP   M=ovccolr0 ACBP=A9
 0003:00000048 00000008 C=DATA     S=.data    G=DGROUP   M=ovcreg   ACBP=A9
 0004:00000000 00000008 C=BSS      S=.bss     G=DGROUP   M=Windows  ACBP=A9
 0004:00000008 0000000C C=BSS      S=.bss     G=DGROUP   M=SysInit  ACBP=A9
 0004:00000014 00000004 C=BSS      S=.bss     G=DGROUP   M=Ovcabot0 ACBP=A9
 0004:00000018 00000004 C=BSS      S=.bss     G=DGROUP   M=ovcaepe  ACBP=A9
 0004:0000001C 00000004 C=BSS      S=.bss     G=DGROUP   M=ovccole0 ACBP=A9
 0004:00000020 00000004 C=BSS      S=.bss     G=DGROUP   M=ovcbtnh0 ACBP=A9
 0004:00000024 00000004 C=BSS      S=.bss     G=DGROUP   M=ovccmdp1 ACBP=A9
 0004:00000028 00000004 C=BSS      S=.bss     G=DGROUP   M=ovccmdp0 ACBP=A9
 0004:0000002C 00000004 C=BSS      S=.bss     G=DGROUP   M=ovccolr0 ACBP=A9
 0004:00000030 00000004 C=BSS      S=.bss     G=DGROUP   M=ovcdock0 ACBP=A9
 0004:00000034 00000008 C=BSS      S=.bss     G=DGROUP   M=Ovcdrpve ACBP=A9
 0004:0000003C 00000004 C=BSS      S=.bss     G=DGROUP   M=OvcEfPe  ACBP=A9
 0004:00000040 00000004 C=BSS      S=.bss     G=DGROUP   M=ovcfnpe  ACBP=A9
 0004:00000044 00000004 C=BSS      S=.bss     G=DGROUP   M=ovcfxfpe ACBP=A9
 0004:00000048 00000004 C=BSS      S=.bss     G=DGROUP   M=ovclbl2  ACBP=A9
 0004:0000004C 00000004 C=BSS      S=.bss     G=DGROUP   M=ovclbl1  ACBP=A9
 0004:00000050 00000004 C=BSS      S=.bss     G=DGROUP   M=ovclbl0  ACBP=A9
 0004:00000054 00000004 C=BSS      S=.bss     G=DGROUP   M=ovclkou1 ACBP=A9
 0004:00000058 00000004 C=BSS      S=.bss     G=DGROUP   M=ovclkou0 ACBP=A9
 0004:0000005C 00000004 C=BSS      S=.bss     G=DGROUP   M=ovcnbk0  ACBP=A9
 0004:00000060 00000004 C=BSS      S=.bss     G=DGROUP   M=OvcNfPe  ACBP=A9
 0004:00000064 00000008 C=BSS      S=.bss     G=DGROUP   M=Ovcoutle ACBP=A9
 0004:0000006C 00000004 C=BSS      S=.bss     G=DGROUP   M=o32vldpe ACBP=A9
 0004:00000070 00000004 C=BSS      S=.bss     G=DGROUP   M=O32IGridEditor1 ACBP=A9
 0004:00000074 00000004 C=BSS      S=.bss     G=DGROUP   M=o32coled ACBP=A9
 0004:00000078 00000004 C=BSS      S=.bss     G=DGROUP   M=O32LobEd ACBP=A9
 0004:0000007C 00000004 C=BSS      S=.bss     G=DGROUP   M=O32IGridItemEd ACBP=A9
 0004:00000080 00000004 C=BSS      S=.bss     G=DGROUP   M=ovcrvped ACBP=A9
 0004:00000084 00000004 C=BSS      S=.bss     G=DGROUP   M=ovcrvced ACBP=A9
 0004:00000088 00000004 C=BSS      S=.bss     G=DGROUP   M=ovctcpe  ACBP=A9
 0004:0000008C 00000004 C=BSS      S=.bss     G=DGROUP   M=ovctbpe2 ACBP=A9
 0004:00000090 00000004 C=BSS      S=.bss     G=DGROUP   M=ovctbpe1 ACBP=A9
 0004:00000094 00000004 C=BSS      S=.bss     G=DGROUP   M=ovcstat0 ACBP=A9
 0004:00000098 00000004 C=BSS      S=.bss     G=DGROUP   M=ovcxfrc1 ACBP=A9
 0004:0000009C 00000004 C=BSS      S=.bss     G=DGROUP   M=ovcxfrc0 ACBP=A9
 0004:000000A0 00000004 C=BSS      S=.bss     G=DGROUP   M=ovcpfpe  ACBP=A9
 0004:000000A4 00000004 C=BSS      S=.bss     G=DGROUP   M=OvcSfPe  ACBP=A9
 0004:000000A8 00000004 C=BSS      S=.bss     G=DGROUP   M=ovcreg   ACBP=A9


  Address             Publics by Name

 0002:000003C0       .O406_d2005..O406_d2005
 0001:000219B8       .O406_d2005.@GetPackageInfoTable
 0001:000219C0       .O406_d2005.@PackageLoad
 0001:000219CC       .O406_d2005.@PackageUnload
 0004:00000074       o32coled..4
 0001:00011378       o32coled..TO32CollectionEditor
 0001:000110A0       o32coled..TO32frmCollEditor
 0001:00011004       o32coled..TProtectedSelectionList
 0001:000120E0       o32coled.Finalization
 0002:00000350       o32coled.o32coled
 0001:00011454       o32coled.ShowO32CollectionEditor
 0001:0001158C       o32coled.TO32CollectionEditor.Edit
 0001:000114E4       o32coled.TO32CollectionEditor.GetAttributes
 0001:000114F0       o32coled.TO32CollectionEditor.GetValue
 0001:00011834       o32coled.TO32frmCollEditor.btnAddClick
 0001:000118D4       o32coled.TO32frmCollEditor.btnDeleteClick
 0001:00011ADC       o32coled.TO32frmCollEditor.btnMoveDownClick
 0001:000119EC       o32coled.TO32frmCollEditor.btnMoveUpClick
 0001:000116E4       o32coled.TO32frmCollEditor.FillGrid
 0001:000116D0       o32coled.TO32frmCollEditor.FormClose
 0001:000115A8       o32coled.TO32frmCollEditor.FormCreate
 0001:000116D4       o32coled.TO32frmCollEditor.FormDestroy
 0001:000115EC       o32coled.TO32frmCollEditor.FormShow
 0001:00011C70       o32coled.TO32frmCollEditor.ListBox1Click
 0001:00011BE0       o32coled.TO32frmCollEditor.ListBox1KeyDown
 0001:00011DD4       o32coled.TO32frmCollEditor.OmPropChange
 0001:00011D54       o32coled.TO32frmCollEditor.SelectComponentList
 0004:00000070       O32IGridEditor1..3
 0001:0000E9CC       O32IGridEditor1..TIGridCmpEd
 0001:0000F0AC       O32IGridEditor1..TO32InspectorGridEditor
 0001:0000F16C       O32IGridEditor1.EditItems
 0001:00010FD4       O32IGridEditor1.Finalization
 0002:00000348       O32IGridEditor1.O32IGridEditor1
 0001:00010FC0       O32IGridEditor1.TIGridCmpEd.ClearImageBtnClick
 0001:00010838       O32IGridEditor1.TIGridCmpEd.Delete1Click
 0001:00010920       O32IGridEditor1.TIGridCmpEd.FormCreate
 0001:00010938       O32IGridEditor1.TIGridCmpEd.FormKeyPress
 0001:0001095C       O32IGridEditor1.TIGridCmpEd.FormShow
 0001:00010774       O32IGridEditor1.TIGridCmpEd.GetChildCount
 0001:00010A70       O32IGridEditor1.TIGridCmpEd.ListItemsKeyDown
 0001:0000F614       O32IGridEditor1.TIGridCmpEd.LoadChildrenOf
 0001:0000FE3C       O32IGridEditor1.TIGridCmpEd.LoadImage
 0001:0000F738       O32IGridEditor1.TIGridCmpEd.LoadItem
 0001:0000F4E0       O32IGridEditor1.TIGridCmpEd.LoadOutline
 0001:0000F284       O32IGridEditor1.TIGridCmpEd.O32FlexButton1Click
 0001:0000F268       O32IGridEditor1.TIGridCmpEd.OkButtonClick
 0001:000109C4       O32IGridEditor1.TIGridCmpEd.OvcSpinner1Click
 0001:0000F4CC       O32IGridEditor1.TIGridCmpEd.SetChange
 0001:00010B78       O32IGridEditor1.TIGridCmpEd.SetItemKeyPress
 0001:00010E2C       O32IGridEditor1.TIGridCmpEd.SetListBoxClickCheck
 0001:00010C88       O32IGridEditor1.TIGridCmpEd.SetListBoxKeyDown
 0001:000107C4       O32IGridEditor1.TIGridCmpEd.TreeView1Change
 0001:00010824       O32IGridEditor1.TIGridCmpEd.TreeView1KeyDown
 0001:00010874       O32IGridEditor1.TIGridCmpEd.TreeView1KeyPress
 0001:00010044       O32IGridEditor1.TIGridCmpEd.UpdateItem
 0001:0000F1BC       O32IGridEditor1.TO32InspectorGridEditor.ExecuteVerb
 0001:0000F218       O32IGridEditor1.TO32InspectorGridEditor.GetVerb
 0001:0000F260       O32IGridEditor1.TO32InspectorGridEditor.GetVerbCount
 0004:0000007C       O32IGridItemEd..4
 0001:0001326C       O32IGridItemEd..TFormIGridItemEditor
 0001:00013544       O32IGridItemEd..TO32IgridCollectionEditor
 0001:000131CC       O32IGridItemEd..TProtectedSelectionList
 0001:00014248       O32IGridItemEd.Finalization
 0002:00000360       O32IGridItemEd.O32IGridItemEd
 0001:00013630       O32IGridItemEd.ShowCollectionEditor
 0001:00013A0C       O32IGridItemEd.TFormIGridItemEditor.btnAddClick
 0001:00013AAC       O32IGridItemEd.TFormIGridItemEditor.btnDeleteClick
 0001:00013C78       O32IGridItemEd.TFormIGridItemEditor.btnMoveDownClick
 0001:00013BC4       O32IGridItemEd.TFormIGridItemEditor.btnMoveUpClick
 0001:000138BC       O32IGridItemEd.TFormIGridItemEditor.FillListBox
 0001:00013784       O32IGridItemEd.TFormIGridItemEditor.FormCreate
 0001:000138AC       O32IGridItemEd.TFormIGridItemEditor.FormDestroy
 0001:000137C8       O32IGridItemEd.TFormIGridItemEditor.FormShow
 0001:00013DD0       O32IGridItemEd.TFormIGridItemEditor.ListBox1Click
 0001:00013D40       O32IGridItemEd.TFormIGridItemEditor.ListBox1KeyDown
 0001:00013F34       O32IGridItemEd.TFormIGridItemEditor.OmPropChange
 0001:00013EB4       O32IGridItemEd.TFormIGridItemEditor.SelectComponentList
 0001:00013768       O32IGridItemEd.TO32IgridCollectionEditor.Edit
 0001:000136C0       O32IGridItemEd.TO32IgridCollectionEditor.GetAttributes
 0001:000136CC       O32IGridItemEd.TO32IgridCollectionEditor.GetValue
 0004:00000078       O32LobEd..3
 0001:000121C0       O32LobEd..TO32frmLkOutEd
 0001:00012110       O32LobEd..TO32LookoutBarEditor
 0001:00013080       O32LobEd.EditLookOut
 0001:0001319C       O32LobEd.Finalization
 0002:00000358       O32LobEd.O32LobEd
 0001:00012FB8       O32LobEd.TO32frmLkOutEd.btnFolderAddClick
 0001:00012F50       O32LobEd.TO32frmLkOutEd.btnFolderDeleteClick
 0001:00012E3C       O32LobEd.TO32frmLkOutEd.btnFolderDownClick
 0001:00012DA4       O32LobEd.TO32frmLkOutEd.btnFolderUpClick
 0001:00013010       O32LobEd.TO32frmLkOutEd.btnItemAddClick
 0001:00012EE8       O32LobEd.TO32frmLkOutEd.btnItemDeleteClick
 0001:00012C30       O32LobEd.TO32frmLkOutEd.btnItemDownClick
 0001:00012B98       O32LobEd.TO32frmLkOutEd.btnItemUpClick
 0001:000126CC       O32LobEd.TO32frmLkOutEd.FormCreate
 0001:00012710       O32LobEd.TO32frmLkOutEd.FormResize
 0001:000128A8       O32LobEd.TO32frmLkOutEd.lbFoldersClick
 0001:00012B18       O32LobEd.TO32frmLkOutEd.lbImagesClick
 0001:00012A60       O32LobEd.TO32frmLkOutEd.lbImagesDrawItem
 0001:00012AC0       O32LobEd.TO32frmLkOutEd.lbItemsClick
 0001:000128F4       O32LobEd.TO32frmLkOutEd.lbItemsDrawItem
 0001:000128D0       O32LobEd.TO32frmLkOutEd.lbItemsMeasureItem
 0001:00012CDC       O32LobEd.TO32frmLkOutEd.PopulateFolderList
 0001:000127B0       O32LobEd.TO32frmLkOutEd.PopulateItemList
 0001:00012634       O32LobEd.TO32LookoutBarEditor.ExecuteVerb
 0001:00012694       O32LobEd.TO32LookoutBarEditor.GetVerb
 0001:000126C4       O32LobEd.TO32LookoutBarEditor.GetVerbCount
 0004:0000006C       o32vldpe..3
 0001:0000DF8C       o32vldpe..TSampleMaskProperty
 0001:0000DD04       o32vldpe..TTO32FrmValidatorExpression
 0001:0000E99C       o32vldpe.Finalization
 0002:00000340       o32vldpe.o32vldpe
 0001:0000E084       o32vldpe.TSampleMaskProperty.AllEqual
 0001:0000E088       o32vldpe.TSampleMaskProperty.Edit
 0001:0000E078       o32vldpe.TSampleMaskProperty.GetAttributes
 0001:0000E880       o32vldpe.TTO32FrmValidatorExpression.FormCreate
 0001:0000E990       o32vldpe.TTO32FrmValidatorExpression.FormDestroy
 0001:0000E8D8       o32vldpe.TTO32FrmValidatorExpression.lbMaskClick
 0004:00000014       Ovcabot0..3
 0001:00001B40       Ovcabot0..TOvcAboutProperty
 0001:00001860       Ovcabot0..TOvcfrmAboutForm
 0001:00001EAC       Ovcabot0.Finalization
 0002:0000022C       Ovcabot0.Ovcabot0
 0001:00001C20       Ovcabot0.TOvcAboutProperty.Edit
 0001:00001C14       Ovcabot0.TOvcAboutProperty.GetAttributes
 0001:00001C74       Ovcabot0.TOvcfrmAboutForm.btnOKClick
 0001:00001C7C       Ovcabot0.TOvcfrmAboutForm.FormCreate
 0001:00001E14       Ovcabot0.TOvcfrmAboutForm.lblGeneralDiscussionClick
 0001:00001D7C       Ovcabot0.TOvcfrmAboutForm.lblHelpClick
 0001:00001CF0       Ovcabot0.TOvcfrmAboutForm.lblTurboLinkClick
 0004:00000018       ovcaepe..5
 0001:000023F8       ovcaepe..TAERangeProperty
 0001:000020FC       ovcaepe..TLocalAE
 0001:00002264       ovcaepe..TLocalEF
 0001:00001EDC       ovcaepe..TOvcfrmAeRange
 0001:00002568       ovcaepe.ChangeFromRange
 0001:000025D0       ovcaepe.ChangeToRange
 0001:00002A48       ovcaepe.Finalization
 0001:00002634       ovcaepe.GetDecimalPlaces
 0002:00000234       ovcaepe.ovcaepe
 0001:000026A4       ovcaepe.TAERangeProperty.Edit
 0001:000024CC       ovcaepe.TAERangeProperty.GetAttributes
 0001:00002510       ovcaepe.TAERangeProperty.GetValue
 0004:00000020       ovcbtnh0..2
 0001:00003CA4       ovcbtnh0..TOvcButtonHeaderEditor
 0001:00003DFC       ovcbtnh0.Finalization
 0002:00000244       ovcbtnh0.ovcbtnh0
 0001:00003D58       ovcbtnh0.TOvcButtonHeaderEditor.ExecuteVerb
 0001:00003DC4       ovcbtnh0.TOvcButtonHeaderEditor.GetVerb
 0001:00003DF4       ovcbtnh0.TOvcButtonHeaderEditor.GetVerbCount
 0004:00000028       ovccmdp0..5
 0001:00004828       ovccmdp0..TOvcCommandProcessorProperty
 0001:00004914       ovccmdp0..TOvcControllerEditor
 0001:00004324       ovccmdp0..TOvcfrmCmdTable
 0001:0000418C       ovccmdp0..TOvcHotEdit
 0003:0000002C       ovccmdp0.cbStates
 0001:00004A80       ovccmdp0.CmdRecToText
 0001:0000615C       ovccmdp0.Finalization
 0001:00004A28       ovccmdp0.GetShortCut
 0001:00004A58       ovccmdp0.KeyToText
 0001:000049C4       ovccmdp0.MakeUserCmdStr
 0002:00000254       ovccmdp0.ovccmdp0
 0001:00004B14       ovccmdp0.TextToKey
 0001:00005FE8       ovccmdp0.TOvcCommandProcessorProperty.Edit
 0001:0000605C       ovccmdp0.TOvcCommandProcessorProperty.GetAttributes
 0001:00006068       ovccmdp0.TOvcControllerEditor.ExecuteVerb
 0001:00006124       ovccmdp0.TOvcControllerEditor.GetVerb
 0001:00006154       ovccmdp0.TOvcControllerEditor.GetVerbCount
 0001:000057B8       ovccmdp0.TOvcfrmCmdTable.AssignKeysToCommand
 0001:000059A0       ovccmdp0.TOvcfrmCmdTable.btnAssignClick
 0001:00005EA0       ovccmdp0.TOvcfrmCmdTable.btnClearClick
 0001:000052CC       ovccmdp0.TOvcfrmCmdTable.btnCloseClick
 0001:000058E8       ovccmdp0.TOvcfrmCmdTable.btnUserCmdClick
 0001:000055B0       ovccmdp0.TOvcfrmCmdTable.ckActiveClick
 0001:000055DC       ovccmdp0.TOvcfrmCmdTable.ckWordstarClick
 0001:00004E8C       ovccmdp0.TOvcfrmCmdTable.CreateEditFields
 0001:00005F98       ovccmdp0.TOvcfrmCmdTable.EditChange
 0001:00005F84       ovccmdp0.TOvcfrmCmdTable.EditEnter
 0001:00004C84       ovccmdp0.TOvcfrmCmdTable.FillListBoxes
 0001:00004E18       ovccmdp0.TOvcfrmCmdTable.FillTabList
 0001:000050B8       ovccmdp0.TOvcfrmCmdTable.FormActivate
 0001:000056EC       ovccmdp0.TOvcfrmCmdTable.FormCreate
 0001:00005738       ovccmdp0.TOvcfrmCmdTable.GetKeys
 0001:0000515C       ovccmdp0.TOvcfrmCmdTable.lbKeysClick
 0001:000053E8       ovccmdp0.TOvcfrmCmdTable.miDeleteClick
 0001:00005BD8       ovccmdp0.TOvcfrmCmdTable.miDuplicateClick
 0001:000052D4       ovccmdp0.TOvcfrmCmdTable.miLoadClick
 0001:00005B20       ovccmdp0.TOvcfrmCmdTable.miNewClick
 0001:00005CF4       ovccmdp0.TOvcfrmCmdTable.miOrderClick
 0001:000054D8       ovccmdp0.TOvcfrmCmdTable.miRenameClick
 0001:00005370       ovccmdp0.TOvcfrmCmdTable.miSaveClick
 0001:000050D4       ovccmdp0.TOvcfrmCmdTable.SetCommandHighlght
 0001:000052B0       ovccmdp0.TOvcfrmCmdTable.TableTabChange
 0001:00004B44       ovccmdp0.TOvcHotEdit.CMDialogChar
 0001:00004C7C       ovccmdp0.TOvcHotEdit.WMChar
 0001:00004B74       ovccmdp0.TOvcHotEdit.WMGetDlgCode
 0001:00004B84       ovccmdp0.TOvcHotEdit.WMKeyDown
 0001:00004C1C       ovccmdp0.TOvcHotEdit.WMSysKeyDown
 0004:00000024       ovccmdp1..2
 0001:00003E2C       ovccmdp1..TOvcfrmScanOrder
 0001:0000415C       ovccmdp1.Finalization
 0002:0000024C       ovccmdp1.ovccmdp1
 0001:000040B8       ovccmdp1.TOvcfrmScanOrder.bntDownClick
 0001:00004070       ovccmdp1.TOvcfrmScanOrder.btnUpClick
 0001:00004118       ovccmdp1.TOvcfrmScanOrder.FormCreate
 0004:0000001C       ovccole0..4
 0001:00002DE0       ovccole0..TOvcCollectionEditor
 0001:00002B08       ovccole0..TOvcfrmCollEditor
 0001:00002A78       ovccole0..TProtectedSelList
 0001:00003C74       ovccole0.Finalization
 0002:0000023C       ovccole0.ovccole0
 0001:00002EBC       ovccole0.ShowCollectionEditor
 0001:00002FF4       ovccole0.TOvcCollectionEditor.Edit
 0001:00002F4C       ovccole0.TOvcCollectionEditor.GetAttributes
 0001:00002F58       ovccole0.TOvcCollectionEditor.GetValue
 0001:000032C8       ovccole0.TOvcfrmCollEditor.btnAddClick
 0001:00003388       ovccole0.TOvcfrmCollEditor.btnDeleteClick
 0001:000035D0       ovccole0.TOvcfrmCollEditor.btnMoveDownClick
 0001:000034B0       ovccole0.TOvcfrmCollEditor.btnMoveUpClick
 0001:00003158       ovccole0.TOvcfrmCollEditor.FillGrid
 0001:00003138       ovccole0.TOvcfrmCollEditor.FormClose
 0001:00003010       ovccole0.TOvcfrmCollEditor.FormCreate
 0001:00003148       ovccole0.TOvcfrmCollEditor.FormDestroy
 0001:00003054       ovccole0.TOvcfrmCollEditor.FormShow
 0001:00003794       ovccole0.TOvcfrmCollEditor.ListBox1Click
 0001:00003704       ovccole0.TOvcfrmCollEditor.ListBox1KeyDown
 0001:00003934       ovccole0.TOvcfrmCollEditor.OmPropChange
 0001:00003908       ovccole0.TOvcfrmCollEditor.SelectComponent
 0001:00003888       ovccole0.TOvcfrmCollEditor.SelectComponentList
 0004:0000002C       ovccolr0..2
 0001:0000618C       ovccolr0..TOvcColorProperty
 0003:00000030       ovccolr0.Colors
 0001:00006420       ovccolr0.Finalization
 0001:00006284       ovccolr0.OrColorToString
 0001:00006370       ovccolr0.OrGetColorValues
 0001:000062EC       ovccolr0.OrStringToColor
 0002:0000025C       ovccolr0.ovccolr0
 0001:000063D8       ovccolr0.TOvcColorProperty.GetValue
 0001:000063F0       ovccolr0.TOvcColorProperty.GetValues
 0001:00006404       ovccolr0.TOvcColorProperty.SetValue
 0004:00000030       ovcdock0..3
 0001:000066B4       ovcdock0..TOvcDockingEditor
 0001:00006450       ovcdock0..TOvcfrmDock
 0001:00006760       ovcdock0.DisplayDockWithDialog
 0001:00006A78       ovcdock0.Finalization
 0002:00000264       ovcdock0.ovcdock0
 0001:00006918       ovcdock0.TOvcDockingEditor.ExecuteVerb
 0001:00006928       ovcdock0.TOvcDockingEditor.GetVerb
 0001:00006954       ovcdock0.TOvcDockingEditor.GetVerbCount
 0001:000069BC       ovcdock0.TOvcfrmDock.btnCancelClick
 0001:000069B0       ovcdock0.TOvcfrmDock.btnOKClick
 0001:0000689C       ovcdock0.TOvcfrmDock.BuildComponentList
 0001:0000695C       ovcdock0.TOvcfrmDock.FormCreate
 0001:000069C8       ovcdock0.TOvcfrmDock.lbComponentListClick
 0001:00006A5C       ovcdock0.TOvcfrmDock.lbComponentListDblClick
 0004:00000038       Ovcdrpve..3
 0001:00006AA8       Ovcdrpve..TOvcfrmRvDataItemEditor
 0001:00006D14       Ovcdrpve..TOvcReportViewItemsProperty
 0001:00007300       Ovcdrpve.Finalization
 0002:0000026C       Ovcdrpve.Ovcdrpve
 0004:00000034       Ovcdrpve.OvcfrmRvDataItemEditor
 0001:0000705C       Ovcdrpve.ShowRvDataItemsEditor
 0001:00006F5C       Ovcdrpve.TOvcfrmRvDataItemEditor.bntAddClick
 0001:0000700C       Ovcdrpve.TOvcfrmRvDataItemEditor.btnDeleteClick
 0001:00006EB8       Ovcdrpve.TOvcfrmRvDataItemEditor.LoadData
 0001:00006DFC       Ovcdrpve.TOvcfrmRvDataItemEditor.OvcDataReportView1Enumerate
 0001:00007038       Ovcdrpve.TOvcfrmRvDataItemEditor.StringGrid1SelectCell
 0001:00006F94       Ovcdrpve.TOvcfrmRvDataItemEditor.StringGrid1SetEditText
 0001:000072DC       Ovcdrpve.TOvcReportViewItemsProperty.Edit
 0001:00007234       Ovcdrpve.TOvcReportViewItemsProperty.GetAttributes
 0001:00007240       Ovcdrpve.TOvcReportViewItemsProperty.GetValue
 0004:0000003C       OvcEfPe..4
 0001:00007730       OvcEfPe..TEfRangeProperty
 0001:0000759C       OvcEfPe..TLocalEF
 0001:00007330       OvcEfPe..TOvcfrmEfRange
 0001:00007890       OvcEfPe.ChangeFromRange
 0001:000078F8       OvcEfPe.ChangeToRange
 0001:00007DE4       OvcEfPe.Finalization
 0001:00007968       OvcEfPe.GetDecimalPlaces
 0002:00000274       OvcEfPe.OvcEfPe
 0001:000079D8       OvcEfPe.TEfRangeProperty.Edit
 0001:00007804       OvcEfPe.TEfRangeProperty.GetAttributes
 0001:00007840       OvcEfPe.TEfRangeProperty.GetValue
 0001:00007DC8       OvcEfPe.TOvcfrmEfRange.DefaultControllerIsSpecialControl
 0001:00007D84       OvcEfPe.TOvcfrmEfRange.FormCreate
 0004:00000040       ovcfnpe..2
 0001:00007E14       ovcfnpe..TOvcFileNameProperty
 0001:00008094       ovcfnpe.Finalization
 0002:0000027C       ovcfnpe.ovcfnpe
 0001:00007F10       ovcfnpe.TOvcFileNameProperty.Edit
 0001:00007EF0       ovcfnpe.TOvcFileNameProperty.GetAttributes
 0001:00007EFC       ovcfnpe.TOvcFileNameProperty.GetValue
 0004:00000044       ovcfxfpe..3
 0001:000080C4       ovcfxfpe..TOvcFixFontNameProperty
 0001:000081A4       ovcfxfpe..TOvcFixFontProperty
 0001:000083D4       ovcfxfpe.Finalization
 0002:00000284       ovcfxfpe.ovcfxfpe
 0001:0000827C       ovcfxfpe.TOvcFixFontNameProperty.GetAttributes
 0001:00008288       ovcfxfpe.TOvcFixFontNameProperty.GetValues
 0001:000082F8       ovcfxfpe.TOvcFixFontProperty.Edit
 0001:000083C8       ovcfxfpe.TOvcFixFontProperty.GetAttributes
 0004:00000050       ovclbl0..4
 0001:000090CC       ovclbl0..TfrmOvcLabel
 0001:000096A4       ovclbl0..TOvcCustomSettingsProperty
 0001:000095FC       ovclbl0..TOvcLabelEditor
 0001:00009788       ovclbl0.EditOvcLabel
 0001:0000B4FC       ovclbl0.Finalization
 0002:00000310       ovclbl0.ovclbl0
 0001:0000B0CC       ovclbl0.TfrmOvcLabel.AppearanceCbChange
 0001:0000B2E4       ovclbl0.TfrmOvcLabel.ColorSchemeCbChange
 0001:0000A784       ovclbl0.TfrmOvcLabel.DeleteBtnClick
 0001:0000A808       ovclbl0.TfrmOvcLabel.DeleteScheme
 0001:00009EA0       ovclbl0.TfrmOvcLabel.FontColorCcbChange
 0001:00009B6C       ovclbl0.TfrmOvcLabel.FontSizeSbChange
 0001:00009EC8       ovclbl0.TfrmOvcLabel.FormCreate
 0001:00009E1C       ovclbl0.TfrmOvcLabel.FromColorCcbChange
 0001:00009CF0       ovclbl0.TfrmOvcLabel.GraduateRgClick
 0001:00009E48       ovclbl0.TfrmOvcLabel.HighlightColorCcbChange
 0001:00009BE8       ovclbl0.TfrmOvcLabel.HighlightDepthSbChange
 0001:0000B028       ovclbl0.TfrmOvcLabel.HighlightDirectionChange
 0001:00009D54       ovclbl0.TfrmOvcLabel.HighlightRgClick
 0001:0000A1C8       ovclbl0.TfrmOvcLabel.SaveAsBtnClick
 0001:0000A890       ovclbl0.TfrmOvcLabel.SchemeCbChange
 0001:0000B080       ovclbl0.TfrmOvcLabel.SchemeChange
 0001:00009E74       ovclbl0.TfrmOvcLabel.ShadowColorCcbChange
 0001:00009C6C       ovclbl0.TfrmOvcLabel.ShadowDepthSbChange
 0001:0000B054       ovclbl0.TfrmOvcLabel.ShadowDirectionChange
 0001:00009DB8       ovclbl0.TfrmOvcLabel.ShadowRgClick
 0001:00009A68       ovclbl0.TOvcCustomSettingsProperty.Edit
 0001:00009B60       ovclbl0.TOvcCustomSettingsProperty.GetAttributes
 0001:000099D8       ovclbl0.TOvcLabelEditor.ExecuteVerb
 0001:00009A30       ovclbl0.TOvcLabelEditor.GetVerb
 0001:00009A60       ovclbl0.TOvcLabelEditor.GetVerbCount
 0004:0000004C       ovclbl1..2
 0001:00008E6C       ovclbl1..TfrmSaveScheme
 0001:0000909C       ovclbl1.Finalization
 0002:00000308       ovclbl1.ovclbl1
 0001:00009058       ovclbl1.TfrmSaveScheme.FormCreate
 0004:00000048       ovclbl2..3
 0001:00008404       ovclbl2..TOvcCustomDirectionPicker
 0001:0000853C       ovclbl2..TOvcDirectionPicker
 0001:00008E3C       ovclbl2.Finalization
 0002:0000028C       ovclbl2.ovclbl2
 0001:00008820       ovclbl2.TOvcCustomDirectionPicker.Create
 0001:00008910       ovclbl2.TOvcCustomDirectionPicker.Destroy
 0001:0000895C       ovclbl2.TOvcCustomDirectionPicker.MouseDown
 0001:00008B1C       ovclbl2.TOvcCustomDirectionPicker.Paint
 0001:00008D50       ovclbl2.TOvcCustomDirectionPicker.SetDirection
 0001:00008E10       ovclbl2.TOvcCustomDirectionPicker.SetDirectionBitmap
 0001:00008DCC       ovclbl2.TOvcCustomDirectionPicker.SetNumDirections
 0001:00008DA0       ovclbl2.TOvcCustomDirectionPicker.SetSelectedBitmap
 0001:00008DF0       ovclbl2.TOvcCustomDirectionPicker.SetShowCenter
 0004:00000058       ovclkou0..2
 0001:0000C438       ovclkou0..TOvcLookoutBarEditor
 0001:0000C5F0       ovclkou0.Finalization
 0002:00000320       ovclkou0.ovclkou0
 0001:0000C4E8       ovclkou0.TOvcLookoutBarEditor.ExecuteVerb
 0001:0000C590       ovclkou0.TOvcLookoutBarEditor.GetVerb
 0001:0000C5E8       ovclkou0.TOvcLookoutBarEditor.GetVerbCount
 0004:00000054       ovclkou1..2
 0001:0000B52C       ovclkou1..TOvcfrmLkOutEd
 0001:0000C2EC       ovclkou1.EditLookOut
 0001:0000C408       ovclkou1.Finalization
 0002:00000318       ovclkou1.ovclkou1
 0001:0000C22C       ovclkou1.TOvcfrmLkOutEd.btnFolderAddClick
 0001:0000C1C4       ovclkou1.TOvcfrmLkOutEd.btnFolderDeleteClick
 0001:0000C0C0       ovclkou1.TOvcfrmLkOutEd.btnFolderDownClick
 0001:0000C038       ovclkou1.TOvcfrmLkOutEd.btnFolderUpClick
 0001:0000C280       ovclkou1.TOvcfrmLkOutEd.btnItemAddClick
 0001:0000C15C       ovclkou1.TOvcfrmLkOutEd.btnItemDeleteClick
 0001:0000BED4       ovclkou1.TOvcfrmLkOutEd.btnItemDownClick
 0001:0000BE4C       ovclkou1.TOvcfrmLkOutEd.btnItemUpClick
 0001:0000B9A0       ovclkou1.TOvcfrmLkOutEd.FormCreate
 0001:0000B9E4       ovclkou1.TOvcfrmLkOutEd.FormResize
 0001:0000BB7C       ovclkou1.TOvcfrmLkOutEd.lbFoldersClick
 0001:0000BDCC       ovclkou1.TOvcfrmLkOutEd.lbImagesClick
 0001:0000BD14       ovclkou1.TOvcfrmLkOutEd.lbImagesDrawItem
 0001:0000BD74       ovclkou1.TOvcfrmLkOutEd.lbItemsClick
 0001:0000BBA8       ovclkou1.TOvcfrmLkOutEd.lbItemsDrawItem
 0001:0000BB84       ovclkou1.TOvcfrmLkOutEd.lbItemsMeasureItem
 0001:0000BF70       ovclkou1.TOvcfrmLkOutEd.PopulateFolderList
 0001:0000BA84       ovclkou1.TOvcfrmLkOutEd.PopulateItemList
 0004:0000005C       ovcnbk0..2
 0001:0000C620       ovcnbk0..TOvcNotebookEditor
 0001:0000C768       ovcnbk0.Finalization
 0002:00000328       ovcnbk0.ovcnbk0
 0001:0000C6C8       ovcnbk0.TOvcNotebookEditor.ExecuteVerb
 0001:0000C734       ovcnbk0.TOvcNotebookEditor.GetVerb
 0001:0000C760       ovcnbk0.TOvcNotebookEditor.GetVerbCount
 0004:00000060       OvcNfPe..3
 0001:0000CA08       OvcNfPe..TNumericMaskProperty
 0001:0000C798       OvcNfPe..TOvcfrmNumericMask
 0001:0000D000       OvcNfPe.Finalization
 0002:00000330       OvcNfPe.OvcNfPe
 0001:0000CAF0       OvcNfPe.TNumericMaskProperty.AllEqual
 0001:0000CAF4       OvcNfPe.TNumericMaskProperty.Edit
 0001:0000CAE4       OvcNfPe.TNumericMaskProperty.GetAttributes
 0001:0000CDA4       OvcNfPe.TOvcfrmNumericMask.FormCreate
 0001:0000CFF4       OvcNfPe.TOvcfrmNumericMask.FormDestroy
 0001:0000CF3C       OvcNfPe.TOvcfrmNumericMask.lbMaskClick
 0004:00000068       Ovcoutle..4
 0001:0000D030       Ovcoutle..TOvcfrmOLItemsEditor
 0001:0000D4D4       Ovcoutle..TOvcOutlineEditor
 0001:0000D3F0       Ovcoutle..TOvcOutlineItemsProperty
 0001:0000DCD4       Ovcoutle.Finalization
 0004:00000064       Ovcoutle.OvcfrmOLItemsEditor
 0002:00000338       Ovcoutle.Ovcoutle
 0001:0000D97C       Ovcoutle.ShowOutlineItemsEditor
 0001:0000D95C       Ovcoutle.TOvcfrmOLItemsEditor.btnApplyClick
 0001:0000D93C       Ovcoutle.TOvcfrmOLItemsEditor.btnDeleteClick
 0001:0000D580       Ovcoutle.TOvcfrmOLItemsEditor.btnNewItemClick
 0001:0000D5FC       Ovcoutle.TOvcfrmOLItemsEditor.btnNewSubItemClick
 0001:0000D914       Ovcoutle.TOvcfrmOLItemsEditor.chkCheckedClick
 0001:0000DC78       Ovcoutle.TOvcfrmOLItemsEditor.edtTextExit
 0001:0000D88C       Ovcoutle.TOvcfrmOLItemsEditor.FormShow
 0001:0000D8B0       Ovcoutle.TOvcfrmOLItemsEditor.OvcOutline1ActiveChange
 0001:0000DC28       Ovcoutle.TOvcfrmOLItemsEditor.OvcSliderEdit1Change
 0001:0000D8C0       Ovcoutle.TOvcfrmOLItemsEditor.rgStyleClick
 0001:0000D64C       Ovcoutle.TOvcfrmOLItemsEditor.SetCurRoot
 0001:0000DB7C       Ovcoutle.TOvcOutlineEditor.ExecuteVerb
 0001:0000DBD8       Ovcoutle.TOvcOutlineEditor.GetVerb
 0001:0000DC20       Ovcoutle.TOvcOutlineEditor.GetVerbCount
 0001:0000DB58       Ovcoutle.TOvcOutlineItemsProperty.Edit
 0001:0000DAB0       Ovcoutle.TOvcOutlineItemsProperty.GetAttributes
 0001:0000DABC       Ovcoutle.TOvcOutlineItemsProperty.GetValue
 0004:000000A0       ovcpfpe..3
 0001:0001E628       ovcpfpe..TOvcfrmPictureMask
 0001:0001E898       ovcpfpe..TPictureMaskProperty
 0001:0001EFA0       ovcpfpe.Finalization
 0002:000003A8       ovcpfpe.ovcpfpe
 0001:0001EC88       ovcpfpe.TOvcfrmPictureMask.FormCreate
 0001:0001EF94       ovcpfpe.TOvcfrmPictureMask.FormDestroy
 0001:0001EEDC       ovcpfpe.TOvcfrmPictureMask.lbMaskClick
 0001:0001E980       ovcpfpe.TPictureMaskProperty.AllEqual
 0001:0001E984       ovcpfpe.TPictureMaskProperty.Edit
 0001:0001E974       ovcpfpe.TPictureMaskProperty.GetAttributes
 0004:000000A8       ovcreg..5
 0001:0001F8A0       ovcreg..TExcludeComponentProperty
 0001:0001F990       ovcreg..TorGenericStringProperty
 0001:0001FB6C       ovcreg..TorRegisteredValidatorsProperty
 0001:0001F720       ovcreg..TOvcHeaderProperty
 0001:0001FD58       ovcreg..TOvcTableEditor
 0001:0001F7F4       ovcreg..TOvcTimerPoolEditor
 0001:00021098       ovcreg.Finalization
 0002:000003B8       ovcreg.ovcreg
 0001:0001FF4C       ovcreg.Register
 0003:00000048       ovcreg.TableVerbs
 0001:0001FCA4       ovcreg.TExcludeComponentProperty.GetValues
 0001:0001FA78       ovcreg.TorGenericStringProperty.GetAttributes
 0001:0001FA84       ovcreg.TorGenericStringProperty.GetValues
 0001:0001FC24       ovcreg.TorRegisteredValidatorsProperty.GetValueList
 0001:0001FDF0       ovcreg.TOvcTableEditor.ExecuteVerb
 0001:0001FF2C       ovcreg.TOvcTableEditor.GetVerb
 0001:0001FF44       ovcreg.TOvcTableEditor.GetVerbCount
 0001:0001FC2C       ovcreg.TOvcTimerPoolEditor.EditProperty
 0004:00000084       ovcrvced..6
 0001:0001557C       ovcrvced..TOvcReportViewEditor
 0001:00015630       ovcrvced..TOvcRvActiveViewProperty
 0001:00015714       ovcrvced..TOvcRvFieldNameProperty
 0001:000157F4       ovcrvced..TOvcRvImgIdxProperty
 0001:000150A8       ovcrvced..TRVCmpEd
 0001:00016C1C       ovcrvced.CopyColumns
 0001:00017098       ovcrvced.EditViews
 0001:00018478       ovcrvced.Finalization
 0002:00000370       ovcrvced.ovcrvced
 0001:000158D0       ovcrvced.Select
 0001:00015904       ovcrvced.SelItem
 0001:00017F8C       ovcrvced.TOvcReportViewEditor.ExecuteVerb
 0001:00017FE8       ovcrvced.TOvcReportViewEditor.GetVerb
 0001:00018038       ovcrvced.TOvcReportViewEditor.GetVerbCount
 0001:00018040       ovcrvced.TOvcRvActiveViewProperty.GetAttributes
 0001:000180A0       ovcrvced.TOvcRvActiveViewProperty.GetValue
 0001:0001804C       ovcrvced.TOvcRvActiveViewProperty.GetValues
 0001:000180B4       ovcrvced.TOvcRvActiveViewProperty.SetValue
 0001:000180BC       ovcrvced.TOvcRvFieldNameProperty.GetAttributes
 0001:00018124       ovcrvced.TOvcRvFieldNameProperty.GetValue
 0001:000180C8       ovcrvced.TOvcRvFieldNameProperty.GetValues
 0001:00018138       ovcrvced.TOvcRvFieldNameProperty.SetValue
 0001:00018294       ovcrvced.TOvcRvImgIdxProperty.GetAttributes
 0001:000182A0       ovcrvced.TOvcRvImgIdxProperty.GetValue
 0001:000182B8       ovcrvced.TOvcRvImgIdxProperty.GetValues
 0001:00018368       ovcrvced.TOvcRvImgIdxProperty.ListDrawValue
 0001:00018438       ovcrvced.TOvcRvImgIdxProperty.ListMeasureHeight
 0001:000183D8       ovcrvced.TOvcRvImgIdxProperty.ListMeasureWidth
 0001:00015BD0       ovcrvced.TRVCmpEd.btnAddClick
 0001:00015A44       ovcrvced.TRVCmpEd.btnAddGClick
 0001:00017C04       ovcrvced.TRVCmpEd.btnCloneClick
 0001:00018140       ovcrvced.TRVCmpEd.btnDeleteClick
 0001:00016230       ovcrvced.TRVCmpEd.btnDownClick
 0001:00017DB0       ovcrvced.TRVCmpEd.btnEditClick
 0001:00017A7C       ovcrvced.TRVCmpEd.btnNewClick
 0001:000168FC       ovcrvced.TRVCmpEd.btnOkClick
 0001:000162FC       ovcrvced.TRVCmpEd.btnPropClick
 0001:00015FF0       ovcrvced.TRVCmpEd.btnRemoveClick
 0001:00016184       ovcrvced.TRVCmpEd.btnUpClick
 0001:000179C8       ovcrvced.TRVCmpEd.cbxNameClick
 0001:00017928       ovcrvced.TRVCmpEd.ClearOldView
 0001:00015E4C       ovcrvced.TRVCmpEd.EnableEdit
 0001:00015ED8       ovcrvced.TRVCmpEd.GListBoxClick
 0001:00017F40       ovcrvced.TRVCmpEd.GListBoxDragDrop
 0001:00017F1C       ovcrvced.TRVCmpEd.GListBoxDragOver
 0001:000176B0       ovcrvced.TRVCmpEd.LoadNewView
 0001:00015F64       ovcrvced.TRVCmpEd.NGListBoxClick
 0001:00017F7C       ovcrvced.TRVCmpEd.NGListBoxDragDrop
 0001:00017F50       ovcrvced.TRVCmpEd.NGListBoxDragOver
 0001:000159C4       ovcrvced.TRVCmpEd.NSListBoxClick
 0001:0001593C       ovcrvced.TRVCmpEd.SListBoxClick
 0001:00016AC0       ovcrvced.UniqueNameFromColumn
 0001:00016F64       ovcrvced.UniqueNameFromTitle
 0001:00016D48       ovcrvced.UpdateColumns
 0004:00000080       ovcrvped..2
 0001:00014278       ovcrvped..TRVCmpEd2
 0001:00014FFC       ovcrvped.Finalization
 0002:00000368       ovcrvped.ovcrvped
 0001:00014EF4       ovcrvped.TRVCmpEd2.cbxSortDirChange
 0001:00014E2C       ovcrvped.TRVCmpEd2.chkAllowResizeClick
 0001:00014C24       ovcrvped.TRVCmpEd2.ChkOwnerDrawClick
 0001:00014DB8       ovcrvped.TRVCmpEd2.chkShowHintClick
 0001:00014BB0       ovcrvped.TRVCmpEd2.chkTotalsClick
 0001:00014E90       ovcrvped.TRVCmpEd2.chkVisibleClick
 0001:00014F58       ovcrvped.TRVCmpEd2.edtAggExit
 0001:00014D58       ovcrvped.TRVCmpEd2.edtColTagChange
 0001:00014CF8       ovcrvped.TRVCmpEd2.edtPrintWidthChange
 0001:00014C98       ovcrvped.TRVCmpEd2.edtWidthChange
 0001:00014734       ovcrvped.TRVCmpEd2.ListBox1Click
 0004:000000A4       OvcSfPe..3
 0001:0001EFD0       OvcSfPe..TOvcfrmSimpleMask
 0001:0001F1EC       OvcSfPe..TSimpleMaskProperty
 0001:0001F6F0       OvcSfPe.Finalization
 0001:0001F368       OvcSfPe.MinI
 0002:000003B0       OvcSfPe.OvcSfPe
 0001:0001F370       OvcSfPe.TOvcfrmSimpleMask.cbxMaskCharacterChange
 0001:0001F2C4       OvcSfPe.TOvcfrmSimpleMask.FormCreate
 0001:0001F4C4       OvcSfPe.TSimpleMaskProperty.AllEqual
 0001:0001F4C8       OvcSfPe.TSimpleMaskProperty.Edit
 0001:0001F4B8       OvcSfPe.TSimpleMaskProperty.GetAttributes
 0004:00000094       ovcstat0..4
 0001:0001A924       ovcstat0..TOvcComponentStateEditor
 0001:0001A534       ovcstat0..TOvcfrmPropsDlg
 0001:0001A9DC       ovcstat0..TStoredPropsProperty
 0001:0001AE34       ovcstat0.BoxCanDropItem
 0001:0001AF30       ovcstat0.BoxDragOver
 0001:0001B028       ovcstat0.BoxMoveFocusedItem
 0001:0001AFD4       ovcstat0.BoxSetItem
 0001:0001AEAC       ovcstat0.DrawItemFocusRect
 0001:0001BFB8       ovcstat0.Finalization
 0002:00000390       ovcstat0.ovcstat0
 0001:0001BA3C       ovcstat0.SetItemIndex
 0001:0001AD08       ovcstat0.ShowStorageDesigner
 0001:0001AAB8       ovcstat0.TOvcComponentStateEditor.ExecuteVerb
 0001:0001ABC4       ovcstat0.TOvcComponentStateEditor.GetVerb
 0001:0001ABF8       ovcstat0.TOvcComponentStateEditor.GetVerbCount
 0001:0001B128       ovcstat0.TOvcfrmPropsDlg.AddButtonClick
 0001:0001B1DC       ovcstat0.TOvcfrmPropsDlg.AddItem
 0001:0001B330       ovcstat0.TOvcfrmPropsDlg.BuildLists
 0001:0001B590       ovcstat0.TOvcfrmPropsDlg.CheckAddItem
 0001:0001B5C8       ovcstat0.TOvcfrmPropsDlg.CheckButtons
 0001:0001B6BC       ovcstat0.TOvcfrmPropsDlg.ClearButtonClick
 0001:0001B6F4       ovcstat0.TOvcfrmPropsDlg.ClearLists
 0001:0001B770       ovcstat0.TOvcfrmPropsDlg.DeleteButtonClick
 0001:0001B78C       ovcstat0.TOvcfrmPropsDlg.DeleteProp
 0001:0001B924       ovcstat0.TOvcfrmPropsDlg.DownBtnClick
 0001:0001B960       ovcstat0.TOvcfrmPropsDlg.FindProp
 0001:0001B9CC       ovcstat0.TOvcfrmPropsDlg.FormCreate
 0001:0001BA10       ovcstat0.TOvcfrmPropsDlg.FormDestroy
 0001:0001BA18       ovcstat0.TOvcfrmPropsDlg.ListClick
 0001:0001BA70       ovcstat0.TOvcfrmPropsDlg.ListToIndex
 0001:0001BAD8       ovcstat0.TOvcfrmPropsDlg.PropertiesListDblClick
 0001:0001BAF8       ovcstat0.TOvcfrmPropsDlg.SetStoredList
 0001:0001BB30       ovcstat0.TOvcfrmPropsDlg.StoredListClick
 0001:0001BB38       ovcstat0.TOvcfrmPropsDlg.StoredListDragDrop
 0001:0001BB90       ovcstat0.TOvcfrmPropsDlg.StoredListDragOver
 0001:0001BBC8       ovcstat0.TOvcfrmPropsDlg.StoredListKeyPress
 0001:0001BBE4       ovcstat0.TOvcfrmPropsDlg.UpBtnClick
 0001:0001BC20       ovcstat0.TOvcfrmPropsDlg.UpdateCurrentClass
 0001:0001BDD8       ovcstat0.TOvcfrmPropsDlg.UpdateCurrentProp
 0001:0001AC00       ovcstat0.TStoredPropsProperty.Edit
 0001:0001ACB0       ovcstat0.TStoredPropsProperty.GetAttributes
 0001:0001ACDC       ovcstat0.TStoredPropsProperty.GetValue
 0004:00000090       ovctbpe1..3
 0001:00019AAC       ovctbpe1..TOvcfrmRowEditor
 0001:00019F90       ovctbpe1..TOvcTableRowProperty
 0001:0001A504       ovctbpe1.Finalization
 0002:00000388       ovctbpe1.ovctbpe1
 0001:0001A0EC       ovctbpe1.TOvcfrmRowEditor.ApplyButtonClick
 0001:0001A4E0       ovctbpe1.TOvcfrmRowEditor.ctlRowNumberChange
 0001:0001A1B8       ovctbpe1.TOvcfrmRowEditor.ctlRowNumberExit
 0001:0001A1D4       ovctbpe1.TOvcfrmRowEditor.ctlUseCustHeightClick
 0001:0001A1EC       ovctbpe1.TOvcfrmRowEditor.ctlUseDefHeightClick
 0001:0001A4D8       ovctbpe1.TOvcfrmRowEditor.DoneButtonClick
 0001:0001A21C       ovctbpe1.TOvcfrmRowEditor.FormShow
 0001:0001A250       ovctbpe1.TOvcfrmRowEditor.RefreshRowData
 0001:0001A364       ovctbpe1.TOvcfrmRowEditor.ResetClick
 0001:0001A390       ovctbpe1.TOvcfrmRowEditor.SetRowNum
 0001:0001A3B8       ovctbpe1.TOvcfrmRowEditor.SetRows
 0001:0001A400       ovctbpe1.TOvcfrmRowEditor.SpeedButton1Click
 0001:0001A424       ovctbpe1.TOvcfrmRowEditor.SpeedButton2Click
 0001:0001A450       ovctbpe1.TOvcfrmRowEditor.SpeedButton3Click
 0001:0001A468       ovctbpe1.TOvcfrmRowEditor.SpeedButton4Click
 0001:0001A488       ovctbpe1.TOvcfrmRowEditor.SpeedButton5Click
 0001:0001A4B8       ovctbpe1.TOvcfrmRowEditor.SpeedButton6Click
 0001:0001A06C       ovctbpe1.TOvcTableRowProperty.Edit
 0001:0001A0E0       ovctbpe1.TOvcTableRowProperty.GetAttributes
 0004:0000008C       ovctbpe2..3
 0001:0001903C       ovctbpe2..TOvcfrmColEditor
 0001:00019460       ovctbpe2..TOvcTableColumnProperty
 0001:00019A7C       ovctbpe2.Finalization
 0002:00000380       ovctbpe2.ovctbpe2
 0001:000195C8       ovctbpe2.TOvcfrmColEditor.AddCellComponentName
 0001:000195D8       ovctbpe2.TOvcfrmColEditor.ApplyButtonClick
 0001:00019A58       ovctbpe2.TOvcfrmColEditor.ctlColNumberChange
 0001:00019684       ovctbpe2.TOvcfrmColEditor.ctlColNumberExit
 0001:000196A8       ovctbpe2.TOvcfrmColEditor.DoneButtonClick
 0001:000196C4       ovctbpe2.TOvcfrmColEditor.FormShow
 0001:000196F4       ovctbpe2.TOvcfrmColEditor.GetCells
 0001:00019820       ovctbpe2.TOvcfrmColEditor.RefreshColData
 0001:000198F4       ovctbpe2.TOvcfrmColEditor.SetColNum
 0001:0001991C       ovctbpe2.TOvcfrmColEditor.SetCols
 0001:00019944       ovctbpe2.TOvcfrmColEditor.SpeedButton1Click
 0001:00019968       ovctbpe2.TOvcfrmColEditor.SpeedButton2Click
 0001:00019998       ovctbpe2.TOvcfrmColEditor.SpeedButton3Click
 0001:000199B0       ovctbpe2.TOvcfrmColEditor.SpeedButton4Click
 0001:000199D4       ovctbpe2.TOvcfrmColEditor.SpeedButton5Click
 0001:00019A08       ovctbpe2.TOvcfrmColEditor.SpeedButton6Click
 0001:00019540       ovctbpe2.TOvcTableColumnProperty.Edit
 0001:000195BC       ovctbpe2.TOvcTableColumnProperty.GetAttributes
 0004:00000088       ovctcpe..5
 0001:000186C8       ovctcpe..TLocalEF
 0001:0001885C       ovctcpe..TLocalTC
 0001:000184A8       ovctcpe..TOvcfrmTCRange
 0001:0001894C       ovctcpe..TTCRangeProperty
 0001:00018ABC       ovctcpe.ChangeFromRange
 0001:00018B24       ovctcpe.ChangeToRange
 0001:0001900C       ovctcpe.Finalization
 0001:00018B94       ovctcpe.GetDecimalPlaces
 0002:00000378       ovctcpe.ovctcpe
 0001:00018C04       ovctcpe.TTCRangeProperty.Edit
 0001:00018A20       ovctcpe.TTCRangeProperty.GetAttributes
 0001:00018A64       ovctcpe.TTCRangeProperty.GetValue
 0004:0000009C       ovcxfrc0..2
 0001:0001E2F4       ovcxfrc0..TOvcTransferEditor
 0001:0001E5F8       ovcxfrc0.Finalization
 0002:000003A0       ovcxfrc0.ovcxfrc0
 0001:0001E3A0       ovcxfrc0.TOvcTransferEditor.ExecuteVerb
 0001:0001E5B8       ovcxfrc0.TOvcTransferEditor.GetVerb
 0001:0001E5F0       ovcxfrc0.TOvcTransferEditor.GetVerbCount
 0004:00000098       ovcxfrc1..2
 0001:0001BFE8       ovcxfrc1..TOvcfrmTransfer
 0001:0001E2C4       ovcxfrc1.Finalization
 0002:00000398       ovcxfrc1.ovcxfrc1
 0001:0001C5BC       ovcxfrc1.Spaces
 0001:0001C578       ovcxfrc1.TOvcfrmTransfer.btnClearAllClick
 0001:0001DFF4       ovcxfrc1.TOvcfrmTransfer.btnCopyToClipboardClick
 0001:0001C5FC       ovcxfrc1.TOvcfrmTransfer.btnGenerateClick
 0001:0001C53C       ovcxfrc1.TOvcfrmTransfer.btnSelectAllClick
 0001:0001C4F0       ovcxfrc1.TOvcfrmTransfer.FormCreate
 0001:0001E29C       ovcxfrc1.TOvcfrmTransfer.NBPageChanged
 0001:0001C5B4       ovcxfrc1.TOvcfrmTransfer.SelectionChange
 0001:0001C378       ovcxfrc1.TOvcfrmTransfer.SetButtonStatus
 0001:0001C3D8       ovcxfrc1.TOvcfrmTransfer.SetInstructionText
 0001:000001F8       ShellAPI.ShellExecute
 0001:000017E4       SysInit.@InitPkg
 0001:00001848       SysInit.@PackageLoad
 0001:00001854       SysInit.@PackageUnload
 0001:000016D4       SysInit.AllocTlsBuffer
 0001:00001790       SysInit.ExitProcessTLS
 0001:00001758       SysInit.ExitThreadTLS
 0001:0000169C       SysInit.FreeLibrary
 0001:000016E0       SysInit.GetTlsSize
 0004:0000000C       SysInit.HInstance
 0001:000017B4       SysInit.InitializeModule
 0001:0000172C       SysInit.InitProcessTLS
 0001:000016E8       SysInit.InitThreadTLS
 0001:000016A4       SysInit.LocalAlloc
 0001:000016AC       SysInit.LocalFree
 0003:00000004       SysInit.Module
 0004:00000008       SysInit.ModuleIsLib
 0004:00000009       SysInit.ModuleIsPackage
 0001:000016B4       SysInit.TlsAlloc
 0004:00000010       SysInit.tlsBuffer
 0001:000016BC       SysInit.TlsFree
 0001:000016C4       SysInit.TlsGetValue
 0003:00000000       SysInit.TlsIndex
 0005:00000000       SysInit.TlsLast
 0003:0000001C       SysInit.TlsProc
 0001:000016CC       SysInit.TlsSetValue
 0001:000017C0       SysInit.UninitializeModule
 0004:00000000       Windows..3
 0001:00000208       Windows.DrawFocusRect
 0001:00000230       Windows.Finalization
 0001:00000200       Windows.FreeLibrary
 0001:00000210       Windows.GetDC
 0001:00000218       Windows.GetFocus
 0004:00000004       Windows.HtmlHelpModule
 0001:00000220       Windows.LoadBitmap
 0001:00000228       Windows.ReleaseDC
 0002:00000008       Windows.Windows


  Address             Publics by Value

 0001:000001F8       ShellAPI.ShellExecute
 0001:00000200       Windows.FreeLibrary
 0001:00000208       Windows.DrawFocusRect
 0001:00000210       Windows.GetDC
 0001:00000218       Windows.GetFocus
 0001:00000220       Windows.LoadBitmap
 0001:00000228       Windows.ReleaseDC
 0001:00000230       Windows.Finalization
 0001:0000169C       SysInit.FreeLibrary
 0001:000016A4       SysInit.LocalAlloc
 0001:000016AC       SysInit.LocalFree
 0001:000016B4       SysInit.TlsAlloc
 0001:000016BC       SysInit.TlsFree
 0001:000016C4       SysInit.TlsGetValue
 0001:000016CC       SysInit.TlsSetValue
 0001:000016D4       SysInit.AllocTlsBuffer
 0001:000016E0       SysInit.GetTlsSize
 0001:000016E8       SysInit.InitThreadTLS
 0001:0000172C       SysInit.InitProcessTLS
 0001:00001758       SysInit.ExitThreadTLS
 0001:00001790       SysInit.ExitProcessTLS
 0001:000017B4       SysInit.InitializeModule
 0001:000017C0       SysInit.UninitializeModule
 0001:000017E4       SysInit.@InitPkg
 0001:00001848       SysInit.@PackageLoad
 0001:00001854       SysInit.@PackageUnload
 0001:00001860       Ovcabot0..TOvcfrmAboutForm
 0001:00001B40       Ovcabot0..TOvcAboutProperty
 0001:00001C14       Ovcabot0.TOvcAboutProperty.GetAttributes
 0001:00001C20       Ovcabot0.TOvcAboutProperty.Edit
 0001:00001C74       Ovcabot0.TOvcfrmAboutForm.btnOKClick
 0001:00001C7C       Ovcabot0.TOvcfrmAboutForm.FormCreate
 0001:00001CF0       Ovcabot0.TOvcfrmAboutForm.lblTurboLinkClick
 0001:00001D7C       Ovcabot0.TOvcfrmAboutForm.lblHelpClick
 0001:00001E14       Ovcabot0.TOvcfrmAboutForm.lblGeneralDiscussionClick
 0001:00001EAC       Ovcabot0.Finalization
 0001:00001EDC       ovcaepe..TOvcfrmAeRange
 0001:000020FC       ovcaepe..TLocalAE
 0001:00002264       ovcaepe..TLocalEF
 0001:000023F8       ovcaepe..TAERangeProperty
 0001:000024CC       ovcaepe.TAERangeProperty.GetAttributes
 0001:00002510       ovcaepe.TAERangeProperty.GetValue
 0001:00002568       ovcaepe.ChangeFromRange
 0001:000025D0       ovcaepe.ChangeToRange
 0001:00002634       ovcaepe.GetDecimalPlaces
 0001:000026A4       ovcaepe.TAERangeProperty.Edit
 0001:00002A48       ovcaepe.Finalization
 0001:00002A78       ovccole0..TProtectedSelList
 0001:00002B08       ovccole0..TOvcfrmCollEditor
 0001:00002DE0       ovccole0..TOvcCollectionEditor
 0001:00002EBC       ovccole0.ShowCollectionEditor
 0001:00002F4C       ovccole0.TOvcCollectionEditor.GetAttributes
 0001:00002F58       ovccole0.TOvcCollectionEditor.GetValue
 0001:00002FF4       ovccole0.TOvcCollectionEditor.Edit
 0001:00003010       ovccole0.TOvcfrmCollEditor.FormCreate
 0001:00003054       ovccole0.TOvcfrmCollEditor.FormShow
 0001:00003138       ovccole0.TOvcfrmCollEditor.FormClose
 0001:00003148       ovccole0.TOvcfrmCollEditor.FormDestroy
 0001:00003158       ovccole0.TOvcfrmCollEditor.FillGrid
 0001:000032C8       ovccole0.TOvcfrmCollEditor.btnAddClick
 0001:00003388       ovccole0.TOvcfrmCollEditor.btnDeleteClick
 0001:000034B0       ovccole0.TOvcfrmCollEditor.btnMoveUpClick
 0001:000035D0       ovccole0.TOvcfrmCollEditor.btnMoveDownClick
 0001:00003704       ovccole0.TOvcfrmCollEditor.ListBox1KeyDown
 0001:00003794       ovccole0.TOvcfrmCollEditor.ListBox1Click
 0001:00003888       ovccole0.TOvcfrmCollEditor.SelectComponentList
 0001:00003908       ovccole0.TOvcfrmCollEditor.SelectComponent
 0001:00003934       ovccole0.TOvcfrmCollEditor.OmPropChange
 0001:00003C74       ovccole0.Finalization
 0001:00003CA4       ovcbtnh0..TOvcButtonHeaderEditor
 0001:00003D58       ovcbtnh0.TOvcButtonHeaderEditor.ExecuteVerb
 0001:00003DC4       ovcbtnh0.TOvcButtonHeaderEditor.GetVerb
 0001:00003DF4       ovcbtnh0.TOvcButtonHeaderEditor.GetVerbCount
 0001:00003DFC       ovcbtnh0.Finalization
 0001:00003E2C       ovccmdp1..TOvcfrmScanOrder
 0001:00004070       ovccmdp1.TOvcfrmScanOrder.btnUpClick
 0001:000040B8       ovccmdp1.TOvcfrmScanOrder.bntDownClick
 0001:00004118       ovccmdp1.TOvcfrmScanOrder.FormCreate
 0001:0000415C       ovccmdp1.Finalization
 0001:0000418C       ovccmdp0..TOvcHotEdit
 0001:00004324       ovccmdp0..TOvcfrmCmdTable
 0001:00004828       ovccmdp0..TOvcCommandProcessorProperty
 0001:00004914       ovccmdp0..TOvcControllerEditor
 0001:000049C4       ovccmdp0.MakeUserCmdStr
 0001:00004A28       ovccmdp0.GetShortCut
 0001:00004A58       ovccmdp0.KeyToText
 0001:00004A80       ovccmdp0.CmdRecToText
 0001:00004B14       ovccmdp0.TextToKey
 0001:00004B44       ovccmdp0.TOvcHotEdit.CMDialogChar
 0001:00004B74       ovccmdp0.TOvcHotEdit.WMGetDlgCode
 0001:00004B84       ovccmdp0.TOvcHotEdit.WMKeyDown
 0001:00004C1C       ovccmdp0.TOvcHotEdit.WMSysKeyDown
 0001:00004C7C       ovccmdp0.TOvcHotEdit.WMChar
 0001:00004C84       ovccmdp0.TOvcfrmCmdTable.FillListBoxes
 0001:00004E18       ovccmdp0.TOvcfrmCmdTable.FillTabList
 0001:00004E8C       ovccmdp0.TOvcfrmCmdTable.CreateEditFields
 0001:000050B8       ovccmdp0.TOvcfrmCmdTable.FormActivate
 0001:000050D4       ovccmdp0.TOvcfrmCmdTable.SetCommandHighlght
 0001:0000515C       ovccmdp0.TOvcfrmCmdTable.lbKeysClick
 0001:000052B0       ovccmdp0.TOvcfrmCmdTable.TableTabChange
 0001:000052CC       ovccmdp0.TOvcfrmCmdTable.btnCloseClick
 0001:000052D4       ovccmdp0.TOvcfrmCmdTable.miLoadClick
 0001:00005370       ovccmdp0.TOvcfrmCmdTable.miSaveClick
 0001:000053E8       ovccmdp0.TOvcfrmCmdTable.miDeleteClick
 0001:000054D8       ovccmdp0.TOvcfrmCmdTable.miRenameClick
 0001:000055B0       ovccmdp0.TOvcfrmCmdTable.ckActiveClick
 0001:000055DC       ovccmdp0.TOvcfrmCmdTable.ckWordstarClick
 0001:000056EC       ovccmdp0.TOvcfrmCmdTable.FormCreate
 0001:00005738       ovccmdp0.TOvcfrmCmdTable.GetKeys
 0001:000057B8       ovccmdp0.TOvcfrmCmdTable.AssignKeysToCommand
 0001:000058E8       ovccmdp0.TOvcfrmCmdTable.btnUserCmdClick
 0001:000059A0       ovccmdp0.TOvcfrmCmdTable.btnAssignClick
 0001:00005B20       ovccmdp0.TOvcfrmCmdTable.miNewClick
 0001:00005BD8       ovccmdp0.TOvcfrmCmdTable.miDuplicateClick
 0001:00005CF4       ovccmdp0.TOvcfrmCmdTable.miOrderClick
 0001:00005EA0       ovccmdp0.TOvcfrmCmdTable.btnClearClick
 0001:00005F84       ovccmdp0.TOvcfrmCmdTable.EditEnter
 0001:00005F98       ovccmdp0.TOvcfrmCmdTable.EditChange
 0001:00005FE8       ovccmdp0.TOvcCommandProcessorProperty.Edit
 0001:0000605C       ovccmdp0.TOvcCommandProcessorProperty.GetAttributes
 0001:00006068       ovccmdp0.TOvcControllerEditor.ExecuteVerb
 0001:00006124       ovccmdp0.TOvcControllerEditor.GetVerb
 0001:00006154       ovccmdp0.TOvcControllerEditor.GetVerbCount
 0001:0000615C       ovccmdp0.Finalization
 0001:0000618C       ovccolr0..TOvcColorProperty
 0001:00006284       ovccolr0.OrColorToString
 0001:000062EC       ovccolr0.OrStringToColor
 0001:00006370       ovccolr0.OrGetColorValues
 0001:000063D8       ovccolr0.TOvcColorProperty.GetValue
 0001:000063F0       ovccolr0.TOvcColorProperty.GetValues
 0001:00006404       ovccolr0.TOvcColorProperty.SetValue
 0001:00006420       ovccolr0.Finalization
 0001:00006450       ovcdock0..TOvcfrmDock
 0001:000066B4       ovcdock0..TOvcDockingEditor
 0001:00006760       ovcdock0.DisplayDockWithDialog
 0001:0000689C       ovcdock0.TOvcfrmDock.BuildComponentList
 0001:00006918       ovcdock0.TOvcDockingEditor.ExecuteVerb
 0001:00006928       ovcdock0.TOvcDockingEditor.GetVerb
 0001:00006954       ovcdock0.TOvcDockingEditor.GetVerbCount
 0001:0000695C       ovcdock0.TOvcfrmDock.FormCreate
 0001:000069B0       ovcdock0.TOvcfrmDock.btnOKClick
 0001:000069BC       ovcdock0.TOvcfrmDock.btnCancelClick
 0001:000069C8       ovcdock0.TOvcfrmDock.lbComponentListClick
 0001:00006A5C       ovcdock0.TOvcfrmDock.lbComponentListDblClick
 0001:00006A78       ovcdock0.Finalization
 0001:00006AA8       Ovcdrpve..TOvcfrmRvDataItemEditor
 0001:00006D14       Ovcdrpve..TOvcReportViewItemsProperty
 0001:00006DFC       Ovcdrpve.TOvcfrmRvDataItemEditor.OvcDataReportView1Enumerate
 0001:00006EB8       Ovcdrpve.TOvcfrmRvDataItemEditor.LoadData
 0001:00006F5C       Ovcdrpve.TOvcfrmRvDataItemEditor.bntAddClick
 0001:00006F94       Ovcdrpve.TOvcfrmRvDataItemEditor.StringGrid1SetEditText
 0001:0000700C       Ovcdrpve.TOvcfrmRvDataItemEditor.btnDeleteClick
 0001:00007038       Ovcdrpve.TOvcfrmRvDataItemEditor.StringGrid1SelectCell
 0001:0000705C       Ovcdrpve.ShowRvDataItemsEditor
 0001:00007234       Ovcdrpve.TOvcReportViewItemsProperty.GetAttributes
 0001:00007240       Ovcdrpve.TOvcReportViewItemsProperty.GetValue
 0001:000072DC       Ovcdrpve.TOvcReportViewItemsProperty.Edit
 0001:00007300       Ovcdrpve.Finalization
 0001:00007330       OvcEfPe..TOvcfrmEfRange
 0001:0000759C       OvcEfPe..TLocalEF
 0001:00007730       OvcEfPe..TEfRangeProperty
 0001:00007804       OvcEfPe.TEfRangeProperty.GetAttributes
 0001:00007840       OvcEfPe.TEfRangeProperty.GetValue
 0001:00007890       OvcEfPe.ChangeFromRange
 0001:000078F8       OvcEfPe.ChangeToRange
 0001:00007968       OvcEfPe.GetDecimalPlaces
 0001:000079D8       OvcEfPe.TEfRangeProperty.Edit
 0001:00007D84       OvcEfPe.TOvcfrmEfRange.FormCreate
 0001:00007DC8       OvcEfPe.TOvcfrmEfRange.DefaultControllerIsSpecialControl
 0001:00007DE4       OvcEfPe.Finalization
 0001:00007E14       ovcfnpe..TOvcFileNameProperty
 0001:00007EF0       ovcfnpe.TOvcFileNameProperty.GetAttributes
 0001:00007EFC       ovcfnpe.TOvcFileNameProperty.GetValue
 0001:00007F10       ovcfnpe.TOvcFileNameProperty.Edit
 0001:00008094       ovcfnpe.Finalization
 0001:000080C4       ovcfxfpe..TOvcFixFontNameProperty
 0001:000081A4       ovcfxfpe..TOvcFixFontProperty
 0001:0000827C       ovcfxfpe.TOvcFixFontNameProperty.GetAttributes
 0001:00008288       ovcfxfpe.TOvcFixFontNameProperty.GetValues
 0001:000082F8       ovcfxfpe.TOvcFixFontProperty.Edit
 0001:000083C8       ovcfxfpe.TOvcFixFontProperty.GetAttributes
 0001:000083D4       ovcfxfpe.Finalization
 0001:00008404       ovclbl2..TOvcCustomDirectionPicker
 0001:0000853C       ovclbl2..TOvcDirectionPicker
 0001:00008820       ovclbl2.TOvcCustomDirectionPicker.Create
 0001:00008910       ovclbl2.TOvcCustomDirectionPicker.Destroy
 0001:0000895C       ovclbl2.TOvcCustomDirectionPicker.MouseDown
 0001:00008B1C       ovclbl2.TOvcCustomDirectionPicker.Paint
 0001:00008D50       ovclbl2.TOvcCustomDirectionPicker.SetDirection
 0001:00008DA0       ovclbl2.TOvcCustomDirectionPicker.SetSelectedBitmap
 0001:00008DCC       ovclbl2.TOvcCustomDirectionPicker.SetNumDirections
 0001:00008DF0       ovclbl2.TOvcCustomDirectionPicker.SetShowCenter
 0001:00008E10       ovclbl2.TOvcCustomDirectionPicker.SetDirectionBitmap
 0001:00008E3C       ovclbl2.Finalization
 0001:00008E6C       ovclbl1..TfrmSaveScheme
 0001:00009058       ovclbl1.TfrmSaveScheme.FormCreate
 0001:0000909C       ovclbl1.Finalization
 0001:000090CC       ovclbl0..TfrmOvcLabel
 0001:000095FC       ovclbl0..TOvcLabelEditor
 0001:000096A4       ovclbl0..TOvcCustomSettingsProperty
 0001:00009788       ovclbl0.EditOvcLabel
 0001:000099D8       ovclbl0.TOvcLabelEditor.ExecuteVerb
 0001:00009A30       ovclbl0.TOvcLabelEditor.GetVerb
 0001:00009A60       ovclbl0.TOvcLabelEditor.GetVerbCount
 0001:00009A68       ovclbl0.TOvcCustomSettingsProperty.Edit
 0001:00009B60       ovclbl0.TOvcCustomSettingsProperty.GetAttributes
 0001:00009B6C       ovclbl0.TfrmOvcLabel.FontSizeSbChange
 0001:00009BE8       ovclbl0.TfrmOvcLabel.HighlightDepthSbChange
 0001:00009C6C       ovclbl0.TfrmOvcLabel.ShadowDepthSbChange
 0001:00009CF0       ovclbl0.TfrmOvcLabel.GraduateRgClick
 0001:00009D54       ovclbl0.TfrmOvcLabel.HighlightRgClick
 0001:00009DB8       ovclbl0.TfrmOvcLabel.ShadowRgClick
 0001:00009E1C       ovclbl0.TfrmOvcLabel.FromColorCcbChange
 0001:00009E48       ovclbl0.TfrmOvcLabel.HighlightColorCcbChange
 0001:00009E74       ovclbl0.TfrmOvcLabel.ShadowColorCcbChange
 0001:00009EA0       ovclbl0.TfrmOvcLabel.FontColorCcbChange
 0001:00009EC8       ovclbl0.TfrmOvcLabel.FormCreate
 0001:0000A1C8       ovclbl0.TfrmOvcLabel.SaveAsBtnClick
 0001:0000A784       ovclbl0.TfrmOvcLabel.DeleteBtnClick
 0001:0000A808       ovclbl0.TfrmOvcLabel.DeleteScheme
 0001:0000A890       ovclbl0.TfrmOvcLabel.SchemeCbChange
 0001:0000B028       ovclbl0.TfrmOvcLabel.HighlightDirectionChange
 0001:0000B054       ovclbl0.TfrmOvcLabel.ShadowDirectionChange
 0001:0000B080       ovclbl0.TfrmOvcLabel.SchemeChange
 0001:0000B0CC       ovclbl0.TfrmOvcLabel.AppearanceCbChange
 0001:0000B2E4       ovclbl0.TfrmOvcLabel.ColorSchemeCbChange
 0001:0000B4FC       ovclbl0.Finalization
 0001:0000B52C       ovclkou1..TOvcfrmLkOutEd
 0001:0000B9A0       ovclkou1.TOvcfrmLkOutEd.FormCreate
 0001:0000B9E4       ovclkou1.TOvcfrmLkOutEd.FormResize
 0001:0000BA84       ovclkou1.TOvcfrmLkOutEd.PopulateItemList
 0001:0000BB7C       ovclkou1.TOvcfrmLkOutEd.lbFoldersClick
 0001:0000BB84       ovclkou1.TOvcfrmLkOutEd.lbItemsMeasureItem
 0001:0000BBA8       ovclkou1.TOvcfrmLkOutEd.lbItemsDrawItem
 0001:0000BD14       ovclkou1.TOvcfrmLkOutEd.lbImagesDrawItem
 0001:0000BD74       ovclkou1.TOvcfrmLkOutEd.lbItemsClick
 0001:0000BDCC       ovclkou1.TOvcfrmLkOutEd.lbImagesClick
 0001:0000BE4C       ovclkou1.TOvcfrmLkOutEd.btnItemUpClick
 0001:0000BED4       ovclkou1.TOvcfrmLkOutEd.btnItemDownClick
 0001:0000BF70       ovclkou1.TOvcfrmLkOutEd.PopulateFolderList
 0001:0000C038       ovclkou1.TOvcfrmLkOutEd.btnFolderUpClick
 0001:0000C0C0       ovclkou1.TOvcfrmLkOutEd.btnFolderDownClick
 0001:0000C15C       ovclkou1.TOvcfrmLkOutEd.btnItemDeleteClick
 0001:0000C1C4       ovclkou1.TOvcfrmLkOutEd.btnFolderDeleteClick
 0001:0000C22C       ovclkou1.TOvcfrmLkOutEd.btnFolderAddClick
 0001:0000C280       ovclkou1.TOvcfrmLkOutEd.btnItemAddClick
 0001:0000C2EC       ovclkou1.EditLookOut
 0001:0000C408       ovclkou1.Finalization
 0001:0000C438       ovclkou0..TOvcLookoutBarEditor
 0001:0000C4E8       ovclkou0.TOvcLookoutBarEditor.ExecuteVerb
 0001:0000C590       ovclkou0.TOvcLookoutBarEditor.GetVerb
 0001:0000C5E8       ovclkou0.TOvcLookoutBarEditor.GetVerbCount
 0001:0000C5F0       ovclkou0.Finalization
 0001:0000C620       ovcnbk0..TOvcNotebookEditor
 0001:0000C6C8       ovcnbk0.TOvcNotebookEditor.ExecuteVerb
 0001:0000C734       ovcnbk0.TOvcNotebookEditor.GetVerb
 0001:0000C760       ovcnbk0.TOvcNotebookEditor.GetVerbCount
 0001:0000C768       ovcnbk0.Finalization
 0001:0000C798       OvcNfPe..TOvcfrmNumericMask
 0001:0000CA08       OvcNfPe..TNumericMaskProperty
 0001:0000CAE4       OvcNfPe.TNumericMaskProperty.GetAttributes
 0001:0000CAF0       OvcNfPe.TNumericMaskProperty.AllEqual
 0001:0000CAF4       OvcNfPe.TNumericMaskProperty.Edit
 0001:0000CDA4       OvcNfPe.TOvcfrmNumericMask.FormCreate
 0001:0000CF3C       OvcNfPe.TOvcfrmNumericMask.lbMaskClick
 0001:0000CFF4       OvcNfPe.TOvcfrmNumericMask.FormDestroy
 0001:0000D000       OvcNfPe.Finalization
 0001:0000D030       Ovcoutle..TOvcfrmOLItemsEditor
 0001:0000D3F0       Ovcoutle..TOvcOutlineItemsProperty
 0001:0000D4D4       Ovcoutle..TOvcOutlineEditor
 0001:0000D580       Ovcoutle.TOvcfrmOLItemsEditor.btnNewItemClick
 0001:0000D5FC       Ovcoutle.TOvcfrmOLItemsEditor.btnNewSubItemClick
 0001:0000D64C       Ovcoutle.TOvcfrmOLItemsEditor.SetCurRoot
 0001:0000D88C       Ovcoutle.TOvcfrmOLItemsEditor.FormShow
 0001:0000D8B0       Ovcoutle.TOvcfrmOLItemsEditor.OvcOutline1ActiveChange
 0001:0000D8C0       Ovcoutle.TOvcfrmOLItemsEditor.rgStyleClick
 0001:0000D914       Ovcoutle.TOvcfrmOLItemsEditor.chkCheckedClick
 0001:0000D93C       Ovcoutle.TOvcfrmOLItemsEditor.btnDeleteClick
 0001:0000D95C       Ovcoutle.TOvcfrmOLItemsEditor.btnApplyClick
 0001:0000D97C       Ovcoutle.ShowOutlineItemsEditor
 0001:0000DAB0       Ovcoutle.TOvcOutlineItemsProperty.GetAttributes
 0001:0000DABC       Ovcoutle.TOvcOutlineItemsProperty.GetValue
 0001:0000DB58       Ovcoutle.TOvcOutlineItemsProperty.Edit
 0001:0000DB7C       Ovcoutle.TOvcOutlineEditor.ExecuteVerb
 0001:0000DBD8       Ovcoutle.TOvcOutlineEditor.GetVerb
 0001:0000DC20       Ovcoutle.TOvcOutlineEditor.GetVerbCount
 0001:0000DC28       Ovcoutle.TOvcfrmOLItemsEditor.OvcSliderEdit1Change
 0001:0000DC78       Ovcoutle.TOvcfrmOLItemsEditor.edtTextExit
 0001:0000DCD4       Ovcoutle.Finalization
 0001:0000DD04       o32vldpe..TTO32FrmValidatorExpression
 0001:0000DF8C       o32vldpe..TSampleMaskProperty
 0001:0000E078       o32vldpe.TSampleMaskProperty.GetAttributes
 0001:0000E084       o32vldpe.TSampleMaskProperty.AllEqual
 0001:0000E088       o32vldpe.TSampleMaskProperty.Edit
 0001:0000E880       o32vldpe.TTO32FrmValidatorExpression.FormCreate
 0001:0000E8D8       o32vldpe.TTO32FrmValidatorExpression.lbMaskClick
 0001:0000E990       o32vldpe.TTO32FrmValidatorExpression.FormDestroy
 0001:0000E99C       o32vldpe.Finalization
 0001:0000E9CC       O32IGridEditor1..TIGridCmpEd
 0001:0000F0AC       O32IGridEditor1..TO32InspectorGridEditor
 0001:0000F16C       O32IGridEditor1.EditItems
 0001:0000F1BC       O32IGridEditor1.TO32InspectorGridEditor.ExecuteVerb
 0001:0000F218       O32IGridEditor1.TO32InspectorGridEditor.GetVerb
 0001:0000F260       O32IGridEditor1.TO32InspectorGridEditor.GetVerbCount
 0001:0000F268       O32IGridEditor1.TIGridCmpEd.OkButtonClick
 0001:0000F284       O32IGridEditor1.TIGridCmpEd.O32FlexButton1Click
 0001:0000F4CC       O32IGridEditor1.TIGridCmpEd.SetChange
 0001:0000F4E0       O32IGridEditor1.TIGridCmpEd.LoadOutline
 0001:0000F614       O32IGridEditor1.TIGridCmpEd.LoadChildrenOf
 0001:0000F738       O32IGridEditor1.TIGridCmpEd.LoadItem
 0001:0000FE3C       O32IGridEditor1.TIGridCmpEd.LoadImage
 0001:00010044       O32IGridEditor1.TIGridCmpEd.UpdateItem
 0001:00010774       O32IGridEditor1.TIGridCmpEd.GetChildCount
 0001:000107C4       O32IGridEditor1.TIGridCmpEd.TreeView1Change
 0001:00010824       O32IGridEditor1.TIGridCmpEd.TreeView1KeyDown
 0001:00010838       O32IGridEditor1.TIGridCmpEd.Delete1Click
 0001:00010874       O32IGridEditor1.TIGridCmpEd.TreeView1KeyPress
 0001:00010920       O32IGridEditor1.TIGridCmpEd.FormCreate
 0001:00010938       O32IGridEditor1.TIGridCmpEd.FormKeyPress
 0001:0001095C       O32IGridEditor1.TIGridCmpEd.FormShow
 0001:000109C4       O32IGridEditor1.TIGridCmpEd.OvcSpinner1Click
 0001:00010A70       O32IGridEditor1.TIGridCmpEd.ListItemsKeyDown
 0001:00010B78       O32IGridEditor1.TIGridCmpEd.SetItemKeyPress
 0001:00010C88       O32IGridEditor1.TIGridCmpEd.SetListBoxKeyDown
 0001:00010E2C       O32IGridEditor1.TIGridCmpEd.SetListBoxClickCheck
 0001:00010FC0       O32IGridEditor1.TIGridCmpEd.ClearImageBtnClick
 0001:00010FD4       O32IGridEditor1.Finalization
 0001:00011004       o32coled..TProtectedSelectionList
 0001:000110A0       o32coled..TO32frmCollEditor
 0001:00011378       o32coled..TO32CollectionEditor
 0001:00011454       o32coled.ShowO32CollectionEditor
 0001:000114E4       o32coled.TO32CollectionEditor.GetAttributes
 0001:000114F0       o32coled.TO32CollectionEditor.GetValue
 0001:0001158C       o32coled.TO32CollectionEditor.Edit
 0001:000115A8       o32coled.TO32frmCollEditor.FormCreate
 0001:000115EC       o32coled.TO32frmCollEditor.FormShow
 0001:000116D0       o32coled.TO32frmCollEditor.FormClose
 0001:000116D4       o32coled.TO32frmCollEditor.FormDestroy
 0001:000116E4       o32coled.TO32frmCollEditor.FillGrid
 0001:00011834       o32coled.TO32frmCollEditor.btnAddClick
 0001:000118D4       o32coled.TO32frmCollEditor.btnDeleteClick
 0001:000119EC       o32coled.TO32frmCollEditor.btnMoveUpClick
 0001:00011ADC       o32coled.TO32frmCollEditor.btnMoveDownClick
 0001:00011BE0       o32coled.TO32frmCollEditor.ListBox1KeyDown
 0001:00011C70       o32coled.TO32frmCollEditor.ListBox1Click
 0001:00011D54       o32coled.TO32frmCollEditor.SelectComponentList
 0001:00011DD4       o32coled.TO32frmCollEditor.OmPropChange
 0001:000120E0       o32coled.Finalization
 0001:00012110       O32LobEd..TO32LookoutBarEditor
 0001:000121C0       O32LobEd..TO32frmLkOutEd
 0001:00012634       O32LobEd.TO32LookoutBarEditor.ExecuteVerb
 0001:00012694       O32LobEd.TO32LookoutBarEditor.GetVerb
 0001:000126C4       O32LobEd.TO32LookoutBarEditor.GetVerbCount
 0001:000126CC       O32LobEd.TO32frmLkOutEd.FormCreate
 0001:00012710       O32LobEd.TO32frmLkOutEd.FormResize
 0001:000127B0       O32LobEd.TO32frmLkOutEd.PopulateItemList
 0001:000128A8       O32LobEd.TO32frmLkOutEd.lbFoldersClick
 0001:000128D0       O32LobEd.TO32frmLkOutEd.lbItemsMeasureItem
 0001:000128F4       O32LobEd.TO32frmLkOutEd.lbItemsDrawItem
 0001:00012A60       O32LobEd.TO32frmLkOutEd.lbImagesDrawItem
 0001:00012AC0       O32LobEd.TO32frmLkOutEd.lbItemsClick
 0001:00012B18       O32LobEd.TO32frmLkOutEd.lbImagesClick
 0001:00012B98       O32LobEd.TO32frmLkOutEd.btnItemUpClick
 0001:00012C30       O32LobEd.TO32frmLkOutEd.btnItemDownClick
 0001:00012CDC       O32LobEd.TO32frmLkOutEd.PopulateFolderList
 0001:00012DA4       O32LobEd.TO32frmLkOutEd.btnFolderUpClick
 0001:00012E3C       O32LobEd.TO32frmLkOutEd.btnFolderDownClick
 0001:00012EE8       O32LobEd.TO32frmLkOutEd.btnItemDeleteClick
 0001:00012F50       O32LobEd.TO32frmLkOutEd.btnFolderDeleteClick
 0001:00012FB8       O32LobEd.TO32frmLkOutEd.btnFolderAddClick
 0001:00013010       O32LobEd.TO32frmLkOutEd.btnItemAddClick
 0001:00013080       O32LobEd.EditLookOut
 0001:0001319C       O32LobEd.Finalization
 0001:000131CC       O32IGridItemEd..TProtectedSelectionList
 0001:0001326C       O32IGridItemEd..TFormIGridItemEditor
 0001:00013544       O32IGridItemEd..TO32IgridCollectionEditor
 0001:00013630       O32IGridItemEd.ShowCollectionEditor
 0001:000136C0       O32IGridItemEd.TO32IgridCollectionEditor.GetAttributes
 0001:000136CC       O32IGridItemEd.TO32IgridCollectionEditor.GetValue
 0001:00013768       O32IGridItemEd.TO32IgridCollectionEditor.Edit
 0001:00013784       O32IGridItemEd.TFormIGridItemEditor.FormCreate
 0001:000137C8       O32IGridItemEd.TFormIGridItemEditor.FormShow
 0001:000138AC       O32IGridItemEd.TFormIGridItemEditor.FormDestroy
 0001:000138BC       O32IGridItemEd.TFormIGridItemEditor.FillListBox
 0001:00013A0C       O32IGridItemEd.TFormIGridItemEditor.btnAddClick
 0001:00013AAC       O32IGridItemEd.TFormIGridItemEditor.btnDeleteClick
 0001:00013BC4       O32IGridItemEd.TFormIGridItemEditor.btnMoveUpClick
 0001:00013C78       O32IGridItemEd.TFormIGridItemEditor.btnMoveDownClick
 0001:00013D40       O32IGridItemEd.TFormIGridItemEditor.ListBox1KeyDown
 0001:00013DD0       O32IGridItemEd.TFormIGridItemEditor.ListBox1Click
 0001:00013EB4       O32IGridItemEd.TFormIGridItemEditor.SelectComponentList
 0001:00013F34       O32IGridItemEd.TFormIGridItemEditor.OmPropChange
 0001:00014248       O32IGridItemEd.Finalization
 0001:00014278       ovcrvped..TRVCmpEd2
 0001:00014734       ovcrvped.TRVCmpEd2.ListBox1Click
 0001:00014BB0       ovcrvped.TRVCmpEd2.chkTotalsClick
 0001:00014C24       ovcrvped.TRVCmpEd2.ChkOwnerDrawClick
 0001:00014C98       ovcrvped.TRVCmpEd2.edtWidthChange
 0001:00014CF8       ovcrvped.TRVCmpEd2.edtPrintWidthChange
 0001:00014D58       ovcrvped.TRVCmpEd2.edtColTagChange
 0001:00014DB8       ovcrvped.TRVCmpEd2.chkShowHintClick
 0001:00014E2C       ovcrvped.TRVCmpEd2.chkAllowResizeClick
 0001:00014E90       ovcrvped.TRVCmpEd2.chkVisibleClick
 0001:00014EF4       ovcrvped.TRVCmpEd2.cbxSortDirChange
 0001:00014F58       ovcrvped.TRVCmpEd2.edtAggExit
 0001:00014FFC       ovcrvped.Finalization
 0001:000150A8       ovcrvced..TRVCmpEd
 0001:0001557C       ovcrvced..TOvcReportViewEditor
 0001:00015630       ovcrvced..TOvcRvActiveViewProperty
 0001:00015714       ovcrvced..TOvcRvFieldNameProperty
 0001:000157F4       ovcrvced..TOvcRvImgIdxProperty
 0001:000158D0       ovcrvced.Select
 0001:00015904       ovcrvced.SelItem
 0001:0001593C       ovcrvced.TRVCmpEd.SListBoxClick
 0001:000159C4       ovcrvced.TRVCmpEd.NSListBoxClick
 0001:00015A44       ovcrvced.TRVCmpEd.btnAddGClick
 0001:00015BD0       ovcrvced.TRVCmpEd.btnAddClick
 0001:00015E4C       ovcrvced.TRVCmpEd.EnableEdit
 0001:00015ED8       ovcrvced.TRVCmpEd.GListBoxClick
 0001:00015F64       ovcrvced.TRVCmpEd.NGListBoxClick
 0001:00015FF0       ovcrvced.TRVCmpEd.btnRemoveClick
 0001:00016184       ovcrvced.TRVCmpEd.btnUpClick
 0001:00016230       ovcrvced.TRVCmpEd.btnDownClick
 0001:000162FC       ovcrvced.TRVCmpEd.btnPropClick
 0001:000168FC       ovcrvced.TRVCmpEd.btnOkClick
 0001:00016AC0       ovcrvced.UniqueNameFromColumn
 0001:00016C1C       ovcrvced.CopyColumns
 0001:00016D48       ovcrvced.UpdateColumns
 0001:00016F64       ovcrvced.UniqueNameFromTitle
 0001:00017098       ovcrvced.EditViews
 0001:000176B0       ovcrvced.TRVCmpEd.LoadNewView
 0001:00017928       ovcrvced.TRVCmpEd.ClearOldView
 0001:000179C8       ovcrvced.TRVCmpEd.cbxNameClick
 0001:00017A7C       ovcrvced.TRVCmpEd.btnNewClick
 0001:00017C04       ovcrvced.TRVCmpEd.btnCloneClick
 0001:00017DB0       ovcrvced.TRVCmpEd.btnEditClick
 0001:00017F1C       ovcrvced.TRVCmpEd.GListBoxDragOver
 0001:00017F40       ovcrvced.TRVCmpEd.GListBoxDragDrop
 0001:00017F50       ovcrvced.TRVCmpEd.NGListBoxDragOver
 0001:00017F7C       ovcrvced.TRVCmpEd.NGListBoxDragDrop
 0001:00017F8C       ovcrvced.TOvcReportViewEditor.ExecuteVerb
 0001:00017FE8       ovcrvced.TOvcReportViewEditor.GetVerb
 0001:00018038       ovcrvced.TOvcReportViewEditor.GetVerbCount
 0001:00018040       ovcrvced.TOvcRvActiveViewProperty.GetAttributes
 0001:0001804C       ovcrvced.TOvcRvActiveViewProperty.GetValues
 0001:000180A0       ovcrvced.TOvcRvActiveViewProperty.GetValue
 0001:000180B4       ovcrvced.TOvcRvActiveViewProperty.SetValue
 0001:000180BC       ovcrvced.TOvcRvFieldNameProperty.GetAttributes
 0001:000180C8       ovcrvced.TOvcRvFieldNameProperty.GetValues
 0001:00018124       ovcrvced.TOvcRvFieldNameProperty.GetValue
 0001:00018138       ovcrvced.TOvcRvFieldNameProperty.SetValue
 0001:00018140       ovcrvced.TRVCmpEd.btnDeleteClick
 0001:00018294       ovcrvced.TOvcRvImgIdxProperty.GetAttributes
 0001:000182A0       ovcrvced.TOvcRvImgIdxProperty.GetValue
 0001:000182B8       ovcrvced.TOvcRvImgIdxProperty.GetValues
 0001:00018368       ovcrvced.TOvcRvImgIdxProperty.ListDrawValue
 0001:000183D8       ovcrvced.TOvcRvImgIdxProperty.ListMeasureWidth
 0001:00018438       ovcrvced.TOvcRvImgIdxProperty.ListMeasureHeight
 0001:00018478       ovcrvced.Finalization
 0001:000184A8       ovctcpe..TOvcfrmTCRange
 0001:000186C8       ovctcpe..TLocalEF
 0001:0001885C       ovctcpe..TLocalTC
 0001:0001894C       ovctcpe..TTCRangeProperty
 0001:00018A20       ovctcpe.TTCRangeProperty.GetAttributes
 0001:00018A64       ovctcpe.TTCRangeProperty.GetValue
 0001:00018ABC       ovctcpe.ChangeFromRange
 0001:00018B24       ovctcpe.ChangeToRange
 0001:00018B94       ovctcpe.GetDecimalPlaces
 0001:00018C04       ovctcpe.TTCRangeProperty.Edit
 0001:0001900C       ovctcpe.Finalization
 0001:0001903C       ovctbpe2..TOvcfrmColEditor
 0001:00019460       ovctbpe2..TOvcTableColumnProperty
 0001:00019540       ovctbpe2.TOvcTableColumnProperty.Edit
 0001:000195BC       ovctbpe2.TOvcTableColumnProperty.GetAttributes
 0001:000195C8       ovctbpe2.TOvcfrmColEditor.AddCellComponentName
 0001:000195D8       ovctbpe2.TOvcfrmColEditor.ApplyButtonClick
 0001:00019684       ovctbpe2.TOvcfrmColEditor.ctlColNumberExit
 0001:000196A8       ovctbpe2.TOvcfrmColEditor.DoneButtonClick
 0001:000196C4       ovctbpe2.TOvcfrmColEditor.FormShow
 0001:000196F4       ovctbpe2.TOvcfrmColEditor.GetCells
 0001:00019820       ovctbpe2.TOvcfrmColEditor.RefreshColData
 0001:000198F4       ovctbpe2.TOvcfrmColEditor.SetColNum
 0001:0001991C       ovctbpe2.TOvcfrmColEditor.SetCols
 0001:00019944       ovctbpe2.TOvcfrmColEditor.SpeedButton1Click
 0001:00019968       ovctbpe2.TOvcfrmColEditor.SpeedButton2Click
 0001:00019998       ovctbpe2.TOvcfrmColEditor.SpeedButton3Click
 0001:000199B0       ovctbpe2.TOvcfrmColEditor.SpeedButton4Click
 0001:000199D4       ovctbpe2.TOvcfrmColEditor.SpeedButton5Click
 0001:00019A08       ovctbpe2.TOvcfrmColEditor.SpeedButton6Click
 0001:00019A58       ovctbpe2.TOvcfrmColEditor.ctlColNumberChange
 0001:00019A7C       ovctbpe2.Finalization
 0001:00019AAC       ovctbpe1..TOvcfrmRowEditor
 0001:00019F90       ovctbpe1..TOvcTableRowProperty
 0001:0001A06C       ovctbpe1.TOvcTableRowProperty.Edit
 0001:0001A0E0       ovctbpe1.TOvcTableRowProperty.GetAttributes
 0001:0001A0EC       ovctbpe1.TOvcfrmRowEditor.ApplyButtonClick
 0001:0001A1B8       ovctbpe1.TOvcfrmRowEditor.ctlRowNumberExit
 0001:0001A1D4       ovctbpe1.TOvcfrmRowEditor.ctlUseCustHeightClick
 0001:0001A1EC       ovctbpe1.TOvcfrmRowEditor.ctlUseDefHeightClick
 0001:0001A21C       ovctbpe1.TOvcfrmRowEditor.FormShow
 0001:0001A250       ovctbpe1.TOvcfrmRowEditor.RefreshRowData
 0001:0001A364       ovctbpe1.TOvcfrmRowEditor.ResetClick
 0001:0001A390       ovctbpe1.TOvcfrmRowEditor.SetRowNum
 0001:0001A3B8       ovctbpe1.TOvcfrmRowEditor.SetRows
 0001:0001A400       ovctbpe1.TOvcfrmRowEditor.SpeedButton1Click
 0001:0001A424       ovctbpe1.TOvcfrmRowEditor.SpeedButton2Click
 0001:0001A450       ovctbpe1.TOvcfrmRowEditor.SpeedButton3Click
 0001:0001A468       ovctbpe1.TOvcfrmRowEditor.SpeedButton4Click
 0001:0001A488       ovctbpe1.TOvcfrmRowEditor.SpeedButton5Click
 0001:0001A4B8       ovctbpe1.TOvcfrmRowEditor.SpeedButton6Click
 0001:0001A4D8       ovctbpe1.TOvcfrmRowEditor.DoneButtonClick
 0001:0001A4E0       ovctbpe1.TOvcfrmRowEditor.ctlRowNumberChange
 0001:0001A504       ovctbpe1.Finalization
 0001:0001A534       ovcstat0..TOvcfrmPropsDlg
 0001:0001A924       ovcstat0..TOvcComponentStateEditor
 0001:0001A9DC       ovcstat0..TStoredPropsProperty
 0001:0001AAB8       ovcstat0.TOvcComponentStateEditor.ExecuteVerb
 0001:0001ABC4       ovcstat0.TOvcComponentStateEditor.GetVerb
 0001:0001ABF8       ovcstat0.TOvcComponentStateEditor.GetVerbCount
 0001:0001AC00       ovcstat0.TStoredPropsProperty.Edit
 0001:0001ACB0       ovcstat0.TStoredPropsProperty.GetAttributes
 0001:0001ACDC       ovcstat0.TStoredPropsProperty.GetValue
 0001:0001AD08       ovcstat0.ShowStorageDesigner
 0001:0001AE34       ovcstat0.BoxCanDropItem
 0001:0001AEAC       ovcstat0.DrawItemFocusRect
 0001:0001AF30       ovcstat0.BoxDragOver
 0001:0001AFD4       ovcstat0.BoxSetItem
 0001:0001B028       ovcstat0.BoxMoveFocusedItem
 0001:0001B128       ovcstat0.TOvcfrmPropsDlg.AddButtonClick
 0001:0001B1DC       ovcstat0.TOvcfrmPropsDlg.AddItem
 0001:0001B330       ovcstat0.TOvcfrmPropsDlg.BuildLists
 0001:0001B590       ovcstat0.TOvcfrmPropsDlg.CheckAddItem
 0001:0001B5C8       ovcstat0.TOvcfrmPropsDlg.CheckButtons
 0001:0001B6BC       ovcstat0.TOvcfrmPropsDlg.ClearButtonClick
 0001:0001B6F4       ovcstat0.TOvcfrmPropsDlg.ClearLists
 0001:0001B770       ovcstat0.TOvcfrmPropsDlg.DeleteButtonClick
 0001:0001B78C       ovcstat0.TOvcfrmPropsDlg.DeleteProp
 0001:0001B924       ovcstat0.TOvcfrmPropsDlg.DownBtnClick
 0001:0001B960       ovcstat0.TOvcfrmPropsDlg.FindProp
 0001:0001B9CC       ovcstat0.TOvcfrmPropsDlg.FormCreate
 0001:0001BA10       ovcstat0.TOvcfrmPropsDlg.FormDestroy
 0001:0001BA18       ovcstat0.TOvcfrmPropsDlg.ListClick
 0001:0001BA3C       ovcstat0.SetItemIndex
 0001:0001BA70       ovcstat0.TOvcfrmPropsDlg.ListToIndex
 0001:0001BAD8       ovcstat0.TOvcfrmPropsDlg.PropertiesListDblClick
 0001:0001BAF8       ovcstat0.TOvcfrmPropsDlg.SetStoredList
 0001:0001BB30       ovcstat0.TOvcfrmPropsDlg.StoredListClick
 0001:0001BB38       ovcstat0.TOvcfrmPropsDlg.StoredListDragDrop
 0001:0001BB90       ovcstat0.TOvcfrmPropsDlg.StoredListDragOver
 0001:0001BBC8       ovcstat0.TOvcfrmPropsDlg.StoredListKeyPress
 0001:0001BBE4       ovcstat0.TOvcfrmPropsDlg.UpBtnClick
 0001:0001BC20       ovcstat0.TOvcfrmPropsDlg.UpdateCurrentClass
 0001:0001BDD8       ovcstat0.TOvcfrmPropsDlg.UpdateCurrentProp
 0001:0001BFB8       ovcstat0.Finalization
 0001:0001BFE8       ovcxfrc1..TOvcfrmTransfer
 0001:0001C378       ovcxfrc1.TOvcfrmTransfer.SetButtonStatus
 0001:0001C3D8       ovcxfrc1.TOvcfrmTransfer.SetInstructionText
 0001:0001C4F0       ovcxfrc1.TOvcfrmTransfer.FormCreate
 0001:0001C53C       ovcxfrc1.TOvcfrmTransfer.btnSelectAllClick
 0001:0001C578       ovcxfrc1.TOvcfrmTransfer.btnClearAllClick
 0001:0001C5B4       ovcxfrc1.TOvcfrmTransfer.SelectionChange
 0001:0001C5BC       ovcxfrc1.Spaces
 0001:0001C5FC       ovcxfrc1.TOvcfrmTransfer.btnGenerateClick
 0001:0001DFF4       ovcxfrc1.TOvcfrmTransfer.btnCopyToClipboardClick
 0001:0001E29C       ovcxfrc1.TOvcfrmTransfer.NBPageChanged
 0001:0001E2C4       ovcxfrc1.Finalization
 0001:0001E2F4       ovcxfrc0..TOvcTransferEditor
 0001:0001E3A0       ovcxfrc0.TOvcTransferEditor.ExecuteVerb
 0001:0001E5B8       ovcxfrc0.TOvcTransferEditor.GetVerb
 0001:0001E5F0       ovcxfrc0.TOvcTransferEditor.GetVerbCount
 0001:0001E5F8       ovcxfrc0.Finalization
 0001:0001E628       ovcpfpe..TOvcfrmPictureMask
 0001:0001E898       ovcpfpe..TPictureMaskProperty
 0001:0001E974       ovcpfpe.TPictureMaskProperty.GetAttributes
 0001:0001E980       ovcpfpe.TPictureMaskProperty.AllEqual
 0001:0001E984       ovcpfpe.TPictureMaskProperty.Edit
 0001:0001EC88       ovcpfpe.TOvcfrmPictureMask.FormCreate
 0001:0001EEDC       ovcpfpe.TOvcfrmPictureMask.lbMaskClick
 0001:0001EF94       ovcpfpe.TOvcfrmPictureMask.FormDestroy
 0001:0001EFA0       ovcpfpe.Finalization
 0001:0001EFD0       OvcSfPe..TOvcfrmSimpleMask
 0001:0001F1EC       OvcSfPe..TSimpleMaskProperty
 0001:0001F2C4       OvcSfPe.TOvcfrmSimpleMask.FormCreate
 0001:0001F368       OvcSfPe.MinI
 0001:0001F370       OvcSfPe.TOvcfrmSimpleMask.cbxMaskCharacterChange
 0001:0001F4B8       OvcSfPe.TSimpleMaskProperty.GetAttributes
 0001:0001F4C4       OvcSfPe.TSimpleMaskProperty.AllEqual
 0001:0001F4C8       OvcSfPe.TSimpleMaskProperty.Edit
 0001:0001F6F0       OvcSfPe.Finalization
 0001:0001F720       ovcreg..TOvcHeaderProperty
 0001:0001F7F4       ovcreg..TOvcTimerPoolEditor
 0001:0001F8A0       ovcreg..TExcludeComponentProperty
 0001:0001F990       ovcreg..TorGenericStringProperty
 0001:0001FA78       ovcreg.TorGenericStringProperty.GetAttributes
 0001:0001FA84       ovcreg.TorGenericStringProperty.GetValues
 0001:0001FB6C       ovcreg..TorRegisteredValidatorsProperty
 0001:0001FC24       ovcreg.TorRegisteredValidatorsProperty.GetValueList
 0001:0001FC2C       ovcreg.TOvcTimerPoolEditor.EditProperty
 0001:0001FCA4       ovcreg.TExcludeComponentProperty.GetValues
 0001:0001FD58       ovcreg..TOvcTableEditor
 0001:0001FDF0       ovcreg.TOvcTableEditor.ExecuteVerb
 0001:0001FF2C       ovcreg.TOvcTableEditor.GetVerb
 0001:0001FF44       ovcreg.TOvcTableEditor.GetVerbCount
 0001:0001FF4C       ovcreg.Register
 0001:00021098       ovcreg.Finalization
 0001:000219B8       .O406_d2005.@GetPackageInfoTable
 0001:000219C0       .O406_d2005.@PackageLoad
 0001:000219CC       .O406_d2005.@PackageUnload
 0002:00000008       Windows.Windows
 0002:0000022C       Ovcabot0.Ovcabot0
 0002:00000234       ovcaepe.ovcaepe
 0002:0000023C       ovccole0.ovccole0
 0002:00000244       ovcbtnh0.ovcbtnh0
 0002:0000024C       ovccmdp1.ovccmdp1
 0002:00000254       ovccmdp0.ovccmdp0
 0002:0000025C       ovccolr0.ovccolr0
 0002:00000264       ovcdock0.ovcdock0
 0002:0000026C       Ovcdrpve.Ovcdrpve
 0002:00000274       OvcEfPe.OvcEfPe
 0002:0000027C       ovcfnpe.ovcfnpe
 0002:00000284       ovcfxfpe.ovcfxfpe
 0002:0000028C       ovclbl2.ovclbl2
 0002:00000308       ovclbl1.ovclbl1
 0002:00000310       ovclbl0.ovclbl0
 0002:00000318       ovclkou1.ovclkou1
 0002:00000320       ovclkou0.ovclkou0
 0002:00000328       ovcnbk0.ovcnbk0
 0002:00000330       OvcNfPe.OvcNfPe
 0002:00000338       Ovcoutle.Ovcoutle
 0002:00000340       o32vldpe.o32vldpe
 0002:00000348       O32IGridEditor1.O32IGridEditor1
 0002:00000350       o32coled.o32coled
 0002:00000358       O32LobEd.O32LobEd
 0002:00000360       O32IGridItemEd.O32IGridItemEd
 0002:00000368       ovcrvped.ovcrvped
 0002:00000370       ovcrvced.ovcrvced
 0002:00000378       ovctcpe.ovctcpe
 0002:00000380       ovctbpe2.ovctbpe2
 0002:00000388       ovctbpe1.ovctbpe1
 0002:00000390       ovcstat0.ovcstat0
 0002:00000398       ovcxfrc1.ovcxfrc1
 0002:000003A0       ovcxfrc0.ovcxfrc0
 0002:000003A8       ovcpfpe.ovcpfpe
 0002:000003B0       OvcSfPe.OvcSfPe
 0002:000003B8       ovcreg.ovcreg
 0002:000003C0       .O406_d2005..O406_d2005
 0003:00000000       SysInit.TlsIndex
 0003:00000004       SysInit.Module
 0003:0000001C       SysInit.TlsProc
 0003:0000002C       ovccmdp0.cbStates
 0003:00000030       ovccolr0.Colors
 0003:00000048       ovcreg.TableVerbs
 0004:00000000       Windows..3
 0004:00000004       Windows.HtmlHelpModule
 0004:00000008       SysInit.ModuleIsLib
 0004:00000009       SysInit.ModuleIsPackage
 0004:0000000C       SysInit.HInstance
 0004:00000010       SysInit.tlsBuffer
 0004:00000014       Ovcabot0..3
 0004:00000018       ovcaepe..5
 0004:0000001C       ovccole0..4
 0004:00000020       ovcbtnh0..2
 0004:00000024       ovccmdp1..2
 0004:00000028       ovccmdp0..5
 0004:0000002C       ovccolr0..2
 0004:00000030       ovcdock0..3
 0004:00000034       Ovcdrpve.OvcfrmRvDataItemEditor
 0004:00000038       Ovcdrpve..3
 0004:0000003C       OvcEfPe..4
 0004:00000040       ovcfnpe..2
 0004:00000044       ovcfxfpe..3
 0004:00000048       ovclbl2..3
 0004:0000004C       ovclbl1..2
 0004:00000050       ovclbl0..4
 0004:00000054       ovclkou1..2
 0004:00000058       ovclkou0..2
 0004:0000005C       ovcnbk0..2
 0004:00000060       OvcNfPe..3
 0004:00000064       Ovcoutle.OvcfrmOLItemsEditor
 0004:00000068       Ovcoutle..4
 0004:0000006C       o32vldpe..3
 0004:00000070       O32IGridEditor1..3
 0004:00000074       o32coled..4
 0004:00000078       O32LobEd..3
 0004:0000007C       O32IGridItemEd..4
 0004:00000080       ovcrvped..2
 0004:00000084       ovcrvced..6
 0004:00000088       ovctcpe..5
 0004:0000008C       ovctbpe2..3
 0004:00000090       ovctbpe1..3
 0004:00000094       ovcstat0..4
 0004:00000098       ovcxfrc1..2
 0004:0000009C       ovcxfrc0..2
 0004:000000A0       ovcpfpe..3
 0004:000000A4       OvcSfPe..3
 0004:000000A8       ovcreg..5
 0005:00000000       SysInit.TlsLast


Bound resource files

Ovcabot0.DFM
ovcaepe.DFM
ovccole0.DFM
ovccmdp1.DFM
ovccmdp0.DFM
ovcdock0.DFM
Ovcdrpve.DFM
OvcEfPe.DFM
ovclbl1.DFM
ovclbl0.DFM
ovclkou1.DFM
OvcNfPe.DFM
Ovcoutle.DFM
o32vldpe.DFM
O32IGridEditor1.DFM
o32coled.DFM
O32LobEd.DFM
O32IGridItemEd.DFM
ovcrvped.DFM
ovcrvced.DFM
ovctcpe.DFM
ovctbpe2.DFM
ovctbpe1.DFM
ovcstat0.DFM
ovcxfrc1.DFM
ovcpfpe.DFM
OvcSfPe.DFM
OVCREG.RES
O406_d2005.res
O406_d2005.drf


Program entry point at 0002:000003C0
